:100000004D424E014D3448300906040001002200E3
:100010006000000000C000000000000000000000C0
:100020000000EEEE000000000000000000000000F4
:1000300001000906000000000000000000000000B0
:100040000200040000002C000000000000B00000CE
:10005000030004002C00300000B00000001000007D
:10006000001C002079000000000000005700000084
:100070000000000000000000000000000000000080
:100080000000000000000000000000000000000070
:10009000000000000000000000000000550000000B
:1000A00029080000090400000108000015080000EC
:1000B00000000000FEE7064B00221A70054B0421E9
:1000C0001A780A431A7080230222DB05FAE7C04639
:1000D0002A00005029000050F0B5A023DB059A68E3
:1000E000A34E0023B37189B07371D2B23371F37030
:1000F000B3707370D12A0BD0D02A01D80132D2B29A
:10010000A023DB059968FF20814311439960F1E743
:10011000984B802212031A6062B6974A0420117825
:100120008143117080220221D205FF311160934971
:10013000FF30088000211170BFF36F8F9048914FFE
:1001400080220538D202BFB280B2178050809180E1
:10015000C046D1888C4A101C5F325E30127800781D
:1001600012020243914201D1884A10E0884B049365
:10017000049B002B02D0049B013BF8E7854B042134
:100180001A780A431A7080230222DB05FAE78248B4
:10019000111D043A0025904202D915600A1CF6E7A9
:1001A0007E4AC021157089005C587D482040585017
:1001B0000221196062B63024013C11D3201C00F0EA
:1001C000D1F90028F8D1E31007220125F3182240C5
:1001D000281C59789040021C0A43D2B25A70EBE7AF
:1001E000704A8023053ADB0292B21F805A800022B7
:1001F0009A80C046DF88BFB2954200D0B0E06A4C1A
:10020000231C3C331A78231C3D331B781B021343F9
:100210009F4204D0B27980231343B371A0E05F4EB4
:10022000012304A8614A33700395011C49CA49C1DE
:1002300012680A60EFF3088301932A1C2B1C5C49A7
:10024000019E081D04398E4204D904AE9E590E60E9
:10025000011CF5E75749019EB1420AD204A81E5875
:100260000868B04203D0002A00D10D1C01220431DD
:10027000F1E70433102BE2D1039500234D48C11858
:100280004D48814204D24D48C05804330860F5E718
:100290003E4B414E191D043B9E4203D9002018607D
:1002A0000B1CF6E7464B03A91A804648920009F05A
:1002B00091FAEFF30882444B191D043B9A4203D98B
:1002C000424818600B1CF7E7414D01235B42381C84
:1002D0002B716B71AB71EB7100F076F93D4A3E48C2
:1002E00016882B1C3D4986420BD0667D1588227DE1
:1002F00036023243954204D10A8892B21A71120A28
:100300005A710A8882421BD0E67DA57D0A88360292
:100310003543AA4214D100250422013AD2B2FF2A61
:1003200007D02F4EA718B65C3F79B742F5D101250B
:10033000F3E7002D04D00A8892B29A71120ADA719A
:100340005A79197912020A4382420FD0DA799979DF
:10035000214B12020A439A4208D000F001FB05E04B
:100360000C4B04211A780A431A70FEE709B0F0BD5D
:100370003009002000E100E02A00005006000040A3
:100380000008000000000000A0070000D4030020C7
:10039000388E000029000050190900202C09002087
:1003A000FF00FFFF00C00000C0BF000094980000E5
:1003B0000400002000000020D0030020109A00005C
:1003C0002E090020D403002090090020CDCDCDCDF2
:1003D00024090020FEAF0000FFFF0000BEBF0000A8
:1003E00000B000008023DB051A79D2B2002A0AD1BE
:1003F00019490A601A89194B92B21A60184B0522E2
:100400001A70184A16E0022A1BD1144A1168842275
:100410009200914202D18722120611E00E4A114940
:100420001068062808D810680968095C09BAD960FC
:1004300013680133136004E0126809688A5C12BA19
:10044000DA60C0468023DB0501221A70C046022212
:100450001A7000221A707047DC030020D0030020BD
:1004600030090020D8030020F8B5384A8025ED0572
:100470002B791278DBB2002A02D1FFF7B3FF63E0D9
:10048000002B0DD1324A33481360334A334913608D
:100490002A89334B92B21A601A6806F079FF49E054
:1004A000012B0FD12B4B1968002943D02A4B2B4A23
:1004B0001868126890423DDA1A68501C18602B7A4E
:1004C0008B5437E0022B30D1224F3B68002B2AD0CF
:1004D0001F4C224922680868214E82420CDA2268A9
:1004E0009B5C1BBAEB6033682068C01880B206F0D2
:1004F000AFFF2368013314E032682368381CD21838
:1005000006F046FF3B68002B0DD0316822688A1840
:1005100032601B781BBAEB60306880B206F098FF3F
:100520000123236006E0EB6004E0032B02D10A4BB9
:1005300000221A60C0468023DB0501221A70C046E3
:1005400002221A7000221A70F8BDC0462C09002041
:10055000DC030020D8030020E0030020E403002097
:10056000D0030020012824D0124A8302D21880230D
:1005700092B2DB021A801A88002801D10E4904E0E9
:100580002F2801D10D4900E00D49521892B25A802E
:1005900000229A80C0462F21DA88081A094B4000B1
:1005A000C15C1818407800020843101A43425841B1
:1005B000C0B2704700000000FB070000FB03000012
:1005C000FF030000A0070000024BDB689872000ADE
:1005D000D872704718030020002934D0012300226C
:1005E00010B488422CD301242407A14204D28142B2
:1005F00002D209011B01F8E7E400A14204D28142C2
:1006000002D249005B00F8E7884201D3401A1A433E
:100610004C08A04202D3001B5C0822438C08A04275
:1006200002D3001B9C082243CC08A04202D3001B2B
:10063000DC082243002803D01B0901D00909E3E7A5
:10064000101C10BC7047002801D00020C04307B424
:10065000024802A14018029003BDC046D900000024
:100660000029F0D003B5FFF7B9FF0EBC4243891A49
:100670001847C046002941D010B4041C4C40A44681
:1006800001230022002900D54942002800D540421C
:1006900088422CD301242407A14204D2814202D2F1
:1006A00009011B01F8E7E400A14204D2814202D211
:1006B00049005B00F8E7884201D3401A1A434C080E
:1006C000A04202D3001B5C0822438C08A04202D344
:1006D000001B9C082243CC08A04202D3001BDC086C
:1006E0002243002803D01B0901D00909E3E7101CAD
:1006F0006446002C00D5404210BC7047002806D04C
:1007000003DB0020C043400801E08020000607B45E
:10071000024802A14018029003BDC0461900000023
:100720000029EBD003B5FFF7A7FF0EBC4243891A9F
:100730001847C0467047C046FFFFFFFFFFFFFFFF9F
:10074000FFFFFFFFFFFFFFFFFFFFFFFFFFFFFFFFB9
:10075000FFFFFFFFFFFFFFFFFFFFFFFFFFFFFFFFA9
:10076000FFFFFFFFFFFFFFFFFFFFFFFFFFFFFFFF99
:10077000FFFFFFFFFFFFFFFFFFFFFFFFFFFFFFFF89
:10078000FFFFFFFFFFFFFFFFFFFFFFFFFFFFFFFF79
:10079000FFFFFFFFFFFFFFFFFFFFFFFFFFFFFFFF69
:1007A000FFFFFFFFFFFFFFFFFFFFFFFFFFFFFFFF59
:1007B000FFFFFFFFFFFFFFFFFFFFFFFFFFFFFFFF49
:1007C000FFFFFFFFFFFFFFFFFFFFFFFFFFFFFFFF39
:1007D000FFFFFFFFFFFFFFFFFFFFFFFFFFFFFFFF29
:1007E000FFFFFFFFFFFFFFFFFFFFFFFFFFFFFFFF19
:1007F000FFFFFFFFFFFFFFFFFFFFFFFFFFFFFFFF09
:1008000083F115E31D1CF9294314406440644064DE
:10081000B882708185D8DFAE5E07B325E676C9560B
:100820001437A4B58737ED446A2F9279A344999C75
:1008300000B32BF8D70E35C8FD0FFAE4F868007145
:100840002191A7270E8DE7932D5B8DCD8B832FFEF6
:10085000B3BC3EF16CF10920743F2AEAFFFF166732
:10086000034B01225A70A0230022DB051A70704747
:1008700020090020034B01229A70A0230022DB05EF
:100880009A7070472009002008B5044B01221A70A5
:10089000034B0022DA7700F091FC08BD200900200C
:1008A00008000050014B18607047C046380900200E
:1008B000014B18687047C04638090020014B18608A
:1008C0007047C0463C090020014B18687047C0467D
:1008D0003C090020014B18687047C0467001002099
:1008E00038B5114C256804F0DBFFA862256804F0D8
:1008F000E9FFE862256804F0F9FF6861256805F002
:1009000025F8A861256805F0E1F808492368096819
:100910001A1CD8320231E861116002221A67C8330A
:1009200003221A6038BDC046700100203C09002037
:1009300008B502F077FE021E05D10749A9230B7105
:1009400006F0B6FCFEE7054B1B6803CB04F05CFC2D
:10095000FFF7C6FF08BDC046CB040020C00300203F
:1009600070B58AB006F09CFB6D460335287008F020
:1009700071FE08F0D1FE02F029FE1E4B0A221B6810
:1009800000269A621022DA6212221A631A4B1A683F
:10099000A4235B00D654FFF7CBFF184B1B88B34250
:1009A00019D001AC311C2322201C08F055FF06236E
:1009B000237001236370124B201C1A782321E270EC
:1009C0001A68E379120A1B0613436360A67006F0E7
:1009D00043FC06F043FB06F063FB041C0E2800D921
:1009E0000E24E0B2074B8200D358291C98472C7084
:1009F000F1E7C046C0030020700100202E0900204E
:100A0000D4030020780100200B4B00221B68322009
:100A1000191DCA670431C86780316420086002204C
:100A2000886001204A60C8604A61CA61A033103101
:100A30000A601A607047C04670010020F7B5214E69
:100A4000019135680090291C943102200C1C0C3C4B
:100A500026680138632E06DD002701262760464000
:100A60008F602F1DFE672768013727608F689742C8
:100A700000D28A600C68012C07DD00240C600C6138
:100A800001272C1C8C34474027600C680E69013408
:100A90000C609E4200D20B6104390028D6D1094F68
:100AA000009C3B68019E1A1DD26F26329200D258DC
:100AB00022801A1C8C32126828329200D35833805C
:100AC000F7BDC04670010020F7B51D1C08AB1C889F
:100AD000194B161C1B680190DA6800915200301CFB
:100AE000002108F0B9FE0123009A1F1C9740002F37
:100AF0000CD00198291C04F0BFFF104B301C1B6860
:100B00000022596906F0FCFF013FF0E7002C0BD1F1
:100B10000720291C04F0B0FF084B2A1C1B685869E9
:100B2000D96906F0A1FD041C301C2B1C0099221C65
:100B300007F028F8201CFEBDC00300207001002033
:100B4000F0B589B0059106920793049006F022FD56
:100B5000264B80791B6802905A699B6905985A4315
:100B60000021920008F078FE029F013F7A1C30D0ED
:100B70001F4B04981A689E235B00D15C04F07CFF35
:100B80001A4B1E6872690192019B013B0393ECD3DF
:100B9000B469184B059AE518039B6343ED18AD0043
:100BA0005519013C13D3B368019A5343E318013339
:100BB000069A9B0098582B6818182860002F04D1BB
:100BC0000299FFF709FD00042860043DE9E7039A54
:100BD000D9E7079B012B07D1054B049800211C681E
:100BE00005F0B2F8FC34A06409B0F0BDC0030020E9
:100BF00070010020FFFFFF3FF0B5524F89B03A6807
:100C0000131C7A331888023BA9281CD97C3211881E
:100C1000062918D81A78052A12D80132D2B21A70C9
:100C20000691494903234B707C235B420590079250
:100C3000CB700020CC2305AA0B7106F039FB04E031
:100C400000221A706BE000221A703C68231C683383
:100C50001B780393002B41D1A16C02910C293DDC40
:100C6000E56B0A2D3ADD666CB31E1E2B1DD81D2DBB
:100C70001BDC236B0193023B3F2B16D8281C311C35
:100C8000FFF7F8FC092810DC0198311CFFF7F2FC93
:100C90000C280ADC0299002917DCA36B002B04D175
:100CA00001991B2901DC132D0FDD331C0D3B1A2B81
:100CB00014D8222D12DC236B293B312B0ED8281C93
:100CC000311CFFF7D7FC022808D0636F052B02DC2C
:100CD0000133636725E00023636720E0039B002561
:100CE0006567AB421DD0E16E05AA0591A36B16495D
:100CF000069303234B707C23246B5B42CB70281C30
:100D000010230B71079406F0D3FA3B68DA6E196F63
:100D10008A4203DC0132DA66281C10E0DD6601201D
:100D20000DE0A36B0949246B05930920642305AAF0
:100D30000B71069406F0BCFA3B680020D86609B037
:100D4000F0BDC04670010020EF010020E801002046
:100D5000F0B51D1C794B93B05B6806909B780791AA
:100D6000580602D5764B01221A7004F09DFE754F8D
:100D7000754C3B68061C196858680A182168986801
:100D80008B690832800092001818002108F064FD79
:100D9000236806985A69191CDB690090301D019080
:100DA0003868303100680630400030180290281C46
:100DB00003F084FA3B6805909A6891001A682368EA
:100DC00001324A435869002108F046FD2068436D0E
:100DD0006430036007F0CEFF2368586900963A68D4
:100DE000191C1268303304325200B6185C312A1CC8
:100DF000019603F0EDFB06F0E5FB061C07F098F802
:100E0000337B002B0CD034300378002B08D12268C0
:100E1000B0235B00D35C022B02D0012004F016FB50
:100E20003B684A495A6818684A709A68CB780870D3
:100E30007F208343802602208A700343764201325A
:100E4000334352000AACCB70AA18532301200B7114
:100E500006F02EFA00212022201C08F0FDFC3B6841
:100E60007F205A68196862709A682170A2700533F1
:100E7000DB7F0221E3706379013283430B4352002D
:100E80001E43AA18667100920022131C0120211C27
:100E900006F00CFA2A4F3B78002B01D102F09AFBA6
:100EA000FFF7AAFE284C2368002812D09B68284927
:100EB0000020089308AADF2309900B7106F0F8F9C7
:100EC000236804209A681B6F02339A4233DC0120A6
:100ED00031E0586904F0AEFE2668301C311C5C31EC
:100EE000303003F057FB23683066186E04F000FEC4
:100EF00004F036FC3B78002B14D1059A002A11D15E
:100F0000144B1A68013A002A01D01A600AE0042240
:100F10001A602368192200923033069807992A1C18
:100F200006F00EFD022004F0B5FA074B1868643095
:100F300007F020FF052013B0F0BDC046F4020020EA
:100F4000A0050020C003002070010020C404002080
:100F5000E801002074010020F0B59400231C0A333E
:100F600085B0DB08DB006946C91A02AF8D4602AACC
:100F7000061C7A60101C0021221C08F06DFC231C4A
:100F80000833DB08DB006946C91A8D4602AD281C10
:100F9000221C002108F060FC0C4C301C2368D96A2C
:100FA0009A6A5C3300910193291C7B6807F004FF67
:100FB000301C02F069FB2368301C9A6ADB6A291C2A
:100FC00000937B6807F0A0F9BD46F7BD70010020D3
:100FD00070B50C1C151C1E1C07F0C6FB0B4B201C0F
:100FE0001B68996ADA6A07F0BBFC201C08F09EF8BF
:100FF000201C07F0B1FD291C321C201C07F04EFEFE
:10100000291C201C03F0CAF870BDC04670010020E6
:1010100038B508F0DBFA051C012008F0EBFA041CD7
:10102000281C03F0ABFF201C03F0B4FF38BD38B51B
:1010300008F0A4FB08F0D2FA051C002008F0DAFA48
:10104000041C281C03F09AFF002004F09DFD201CC6
:1010500003F0A0FF04F0DCF938BD10B5A4B08C2279
:10106000041C002101A808F0F7FB01A8211C07F0CF
:1010700055FE07F07DFE01A8211C02F06FFB24B095
:1010800010BD0000F7B5071C06F052FF474E34684C
:101090002379002B02D0012B28D061E0444A211C87
:1010A0001268FC3112784D6C016C2260002905DC5D
:1010B0002169404B994202D0236901332361032106
:1010C0004A432369521093424ADD436C002B47D1B7
:1010D000221C7E321370391CA2690420FFF730FDF8
:1010E000326862210123FF3153542CE0304B271C1E
:1010F0001B68FC3701935B78BD6C23602069AE23CD
:101100005B000130E15AFFF70BFB002904D1236992
:10111000002B01DD7B6CED186023FF33E35C012BBA
:1011200009D1019A62211378FF31236002237D6C7B
:101130006354002307E022691E4B9A4210D02369B2
:10114000013323610CE0316860200022FF300A5433
:101150000B710A6118490E33101C0B7106F0A8F8C8
:101160003368186804F068FF041C281C04F088FF2A
:10117000241A0120002C08DD3368186804F05CFF95
:10118000041C281C04F07CFF201A32686221FF3105
:10119000535C012B04D162210020FF315054181CF4
:1011A00004F054F904F05EF9F7BDC0467001002068
:1011B0003C090020FFFFFF7FCB04002070B52A4DC3
:1011C000B0222B6852009A5C012A01D1274E01E01F
:1011D000B0263603B2246400195B00291CD0B32268
:1011E00052009A5C002A01D000220BE01B5B052B09
:1011F0000AD8301C04F02AF904F046F92B681A5B6F
:10120000013292B21A532EE0BFF34F8F184A194B96
:101210001A60BFF34F8FFEE7012A14D11A79012A11
:1012200009D16022FF329A5C002A0CD19E22520022
:10123000995C042005E0002A05D19E225200995CA9
:10124000022004F0C5FAB3232A685B00D35C002BAC
:1012500009D1301C04F0FAF804F016F901212A68CB
:10126000B2238B40D15270BD70010020FFFFFF0000
:101270000400FA050CED00E0F8B5071C0E1C151C67
:101280001C1C9A420DD0074B1B681B193933FF33C6
:10129000587906F067F8381C311C2A1C231C06F00C
:1012A00013FBF8BD70010020F0B58DB005AE041C35
:1012B0000F1C0C220021301C08F0CEFA2C4D062207
:1012C000291C03A808F086FA08F058FAA30003A91D
:1012D000640009199F5101910024019B6F461D5D17
:1012E000002110220A3708A808F0B6FA391C02AA11
:1012F00008AB281C04F02CFE00217A5E05AEAB0082
:1013000001349A51022CE8D11949032706313A1CBD
:1013100008A808F05FFA174C0123E3700020EB23C4
:10132000211C08AA2371677005F0C2FF7C235B4271
:10133000E3700020EC23211C321C2371677005F040
:10134000B7FF33680020182B0FDD0B495A185142A4
:101350004A41524215407268934201DD131C012537
:10136000B268934200DD0225281C0DB0F0BDC046D6
:10137000A4980000EF01002001000080F0B587B0C4
:1013800006F020F9029006F0D3FD016CAE4D002965
:1013900006D1846C631E9C41E4B2002C05D000E0B1
:1013A00001242B680022B03305E02B68B0331A68A3
:1013B000FE2A01DC01321A602B68191CC4310A882C
:1013C000181C0392AC3000220A80027019390A7886
:1013D000D2B2002A08D00B785BB2022B00D00123D6
:1013E000037000230B702AE11E1CA8363778002FEB
:1013F0000AD0012404700A70191CA931B433327068
:10140000271C0A701A601BE1002C4ED11A1CB43242
:10141000116800291FDD4B1E8C491360201C0493AA
:1014200004AA14230B71059405F042FF2B68B43312
:101430001E68012E39D186491523221C201C0B71F0
:1014400005F036FF2B68371C1A1CB4321460AC331D
:1014500003221A70F4E01A1CD832126811887D4AEF
:10146000914222D01A1CC03211887B4A12685288DD
:101470008A421AD8794E3068027C181CB030006855
:10148000904212DB04AA1180C2331B887449538036
:1014900002234B70CB70201C15230B7105F008FF45
:1014A00032682B68527CB4331A606C4E33685F7DAF
:1014B000002F00D0C3E0644D002C24D12A680133F2
:1014C000BC32DB7F12689A4215DB61491223201C73
:1014D000221C0B7105F0ECFE2A683068131CB8332F
:1014E0001968023001311960C07F814203DB1C6042
:1014F000AC32022313702A680023111CAA31BC32BB
:101500000B7013603CE02B681A1CB4321760203259
:101510001278002A34D01A1CC232C03312881B88B9
:101520004A49049305921923381C04AA0B7105F04B
:10153000BFFE2B683268191CC0310D88D08B16395C
:10154000854215D2181CC2300588508D85420FD2B5
:10155000D08D039D85420BDA0978002910D1BC3368
:1015600001321968D27F91420ADA0131196007E02D
:1015700001220A70191C0022BC31B8330A601A60BB
:10158000314D2B681A1CD4321278002A58D1029897
:10159000027B002A4FD01A1CA8321278002A4FD1A1
:1015A0002E4E186B33683268DB8A518B928B029314
:1015B00033681B8B0093029B05F0A5FF33680290F4
:1015C000DB8C2A689C463368106B1B8D3268518C0B
:1015D000928C0093634605F096FF2B681A1CC0326C
:1015E0001188029AC233914207DA1A88824204DAD9
:1015F00032680398928D904210DB04AA11801B88F8
:101600001749538002234B70CB70002017230B71B6
:1016100005F04EFE2B680122A9331A702B681A1CA4
:10162000A9321278002A0BD0002C09D0A83301224D
:101630001A70002704E0A9331A70171C00E0012774
:10164000381C07B0F0BDC04670010020E801002042
:10165000CB040020FFFF00003C09002038090020D7
:10166000EF010020F0B58FB000AFF960061C03F069
:1016700097FC786103F088FC9D4D78602C68684683
:10168000E268131C0E33DB08DB00C01A8546606875
:101690006B461218FB62131C0E33DB086946DB0035
:1016A000C91A53000E33DB08DB008D46C91A6846A1
:1016B00079628D460021786308F0CEF8E0686168B1
:1016C0004218012152004942786A08F0C5F8E268E0
:1016D000012152004942F86808F0BEF82B68F86A08
:1016E000DA68796908F076F8002E14D1804D814CC3
:1016F0002B6808201A681B7922706370A3707F23FF
:101700005B42E370211CD223FA6A237105F0D0FDFD
:101710002B681B68C0E040240025FC61BD620122EB
:10172000F86A002104F0F6FD0320002104F0A4F97A
:101730006F4C704923681E6858689A680423CB7000
:1017400051230B716C4B8A701B6801325B699200EC
:1017500048709A1802200E7005F0AAFD23681B68D5
:101760003B633E6B624B013EBE6100D284E01B686E
:101770005E68013E00D27CE05D4B3C6B1B68B86943
:1017800099685B6861435C4A434312687118526907
:101790000131FC6889009B1989585A009446221C23
:1017A0008DB262443D6215888CB23D602DB2A54277
:1017B00005DC3D68601B7C6A6546605322E0786A00
:1017C000041C64443C610025645F013415D07D6BCA
:1017D000EC18257868B2B860013001DA013503E011
:1017E000B868002809DD013D02235B4225701380A3
:1017F000BB6A01339BB2BB622DE07D6BEC18257890
:10180000002D01D111800DE06DB2681C06D13A6A3D
:1018100039683D69881A2880002202E0012D01D133
:10182000FF2222707C6BE1180A7850B2002806DC97
:101830007D6A6446285F013007D0002A05D1FC6A22
:101840000132E3563E2B05DD05E0FD6AEB56002B29
:1018500001DD013A0A70264BB8691B687C6B5B6836
:101860007D6943439B19E15CEA5CFC6A8A18E25497
:101870007FE7BD693D6374E71B68BC6ADA681B6972
:10188000D3189C4200DB31E7FB69013BDBB2FB6113
:10189000002B00D043E729E7013B11D32A685268A7
:1018A000013AF9D32968FE6A4968594389187118C1
:1018B0007E68F0183E300E78007830180870EFE738
:1018C000F86A0021012204F025FD2B68211C18680C
:1018D0001B7920706370A3707F235B42E370082044
:1018E0001D23FA6A237105F0E3FCBD460FB0F0BD7D
:1018F000C0030020C40400207001002038B5051C7E
:101900000C1C03F041FB34300078211C4342584149
:101910002840FFF7A7FE38BDF0B585B0051C019142
:1019200007F02CFF174F19230393391CFE2302AA3B
:1019300000203B71029505F0BBFC134E9E243268DB
:101940006400105D291CFFF7AFFC104B051C1B68E1
:101950000199D86833681A5D2B1CFFF78DFC291C90
:10196000022004F089F832680020135D391C0293CC
:1019700002AAE6233B71039505F09AFC33681D55D6
:1019800005B0F0BDE801002070010020C003002078
:10199000F0B5534E89B000AFF960336851491A1C55
:1019A0008D446946FC32D1664E49B0248D44694667
:1019B0003861116764001B5D0125002B02D005F022
:1019C00085FB051C3268135D474CAB422ED0236863
:1019D000012D10D10A2199621021D96212211963B7
:1019E000A42300215B00D15407F034FE07F094FEDD
:1019F000FEF79EFF14E002221A629A62062200217C
:101A0000DA62082219611A6305F0C4FD002202732C
:101A100007F078FE236803CB03F0F6FBFEF760FFC8
:101A20003268B0235B00D55404F01AF92468694683
:101A3000E369E2689E00331C0A33DB08DB00C91A45
:101A40008D466B46FB6153000833DB08DB00C91A87
:101A5000D31DDB08DB00B9608D46C91A8D4679605D
:101A60006846002107F0F8FEA46A6A46E5002B1CD0
:101A7000A4000833D21A231C0833DB08DB00954688
:101A80006946D21A9546B9617A61F869321C00211B
:101A900007F0E2FE2A1CB869002107F0DDFE221CD7
:101AA0007869002107F0D8FE104B7A68B9685A604F
:101AB00000221960DA60F969BA6999601A61796976
:101AC000074A59611168B02252008A5C08499000A7
:101AD00044583869F968A047BD4609B0F0BDC04612
:101AE0007001002058FDFFFFC003002040090020C6
:101AF000B401002010B5041C05F03AFB05F0D0FA43
:101B0000A042FBD007F082FDFEF712FF05F068F956
:101B100010BD0000F0B587B002AF051CFFF778FAE2
:101B2000FEF7D2FE3A4B041C1B685B887B6005F015
:101B30005BFA6B4600203B6004F026F803F0ECFFF4
:101B4000344E336833331B78002B1ED0324B0022C7
:101B50001B68628039331978381C4900013108301C
:101B600005F0BFFC03F010FE2C4B1A689E235B00AF
:101B7000D35C3268D218927C019382180095D2B25D
:101B8000B868F968002300F0E1FC03F005FEC0B27C
:101B900005F0E8FBFEF7A4FE214B6A461B68012016
:101BA000DB685B000833DB08DB00D21A954602A92C
:101BB000FFF7A4FE3B689D4605F0DAFA05F0E2FA6D
:101BC000052818D004D8002817D0032810D80CE016
:101BD0000B280AD004D806280FD103F019FC0CE01A
:101BE000031C113BDBB2022B07D801F07FFA04E0A3
:101BF00004F078FF01E003F0F9FB05F051FAA84288
:101C0000DCD0FFF714FA7A68BD46628005B0F0BDFB
:101C10003C090020380900205C09002070010020E8
:101C2000C003002098B500AF041C05F0A1FA0A4BD0
:101C30006A461B680120DB685B000833DB08DB00B9
:101C4000D21A95466946FFF759FE05F029FAA042D7
:101C5000FBD0BD4698BDC046C003002010B5041C93
:101C600005F086FA01F041FA05F01AFAA042FBD01D
:101C700010BD10B5041C05F07BFA04F07BF805F0EC
:101C80000FFAA042FBD010BD1FB5041C05F070FA7E
:101C9000104B02A81B68393319784900013105F04F
:101CA00020FC03F071FD0C4B03991A689E235B0026
:101CB000D35C0A4A1268D218927C01938218D2B27D
:101CC00000940298022300F041FC05F0E9F9A042DB
:101CD000FBD01FBD5C0900207001002038090020E6
:101CE0001FB5041C05F044FA104B02A81B683933D9
:101CF00019784900013105F0F4FB03F045FD0C4B68
:101D000003991A689E235B00D35C0A4A1268D218B2
:101D1000927C01938218D2B200940298012300F0C1
:101D200015FC05F0BDF9A042FBD01FBD5C090020E9
:101D3000700100203809002010B5041C05F018FAC5
:101D40000220002103F098FE03F0DEFB01200021B9
:101D500003F092FE03F026FF05F0A2F9A042FBD0AB
:101D600010BD10B5041C05F003FA002003F03EFA84
:101D70000220002103F080FE03F0C6FB01200021B9
:101D800003F07AFE03F00EFF05F08AF9A042FBD0C3
:101D9000012003F02BFA10BDF0B5A3B002AF3861FB
:101DA00005F0E6F9002007F0E3FC07F0B5FC0020A1
:101DB00003F0EAFE5F4C694623685D6818681B699A
:101DC0004543EB180733DB08DB00C91A8D4602AA2E
:101DD000FA6103F0E5F803F0D7F8FB695D19181C08
:101DE000291C7D6104F08EF823686C465A681B69D3
:101DF000D3189B000A33DB08DB00E41AA54602ACCB
:101E0000BC6105F0B5F9381C00212022203007F014
:101E100023FD484D20202B68212419681A79C155CB
:101E20002220C255E2550533DB7F23212522CB55E5
:101E3000D35D7F220124F969934323432520C355B1
:101E400000220091391C131C0420203105F02EFAC9
:101E5000221CF869796904F05DFA0220002103F080
:101E60000BFE03F051FB201C002103F005FE2D6842
:101E7000314B6E682A691968BB69B4001C19921944
:101E80009446BC60002363450CDA9A00B34203DA3F
:101E9000CC69B869A45802E04C6AB868A458845068
:101EA0000133F0E73C1C4034201C0021202207F0C5
:101EB000D3FC2968AB6821706670A3700535EA7F92
:101EC0007F26E27062790425B2432A4362711A4A7E
:101ED000013312689B005269211CD3180022203460
:101EE00000930220131C05F0E1F9201C00212022A0
:101EF00007F0B2FC012323700E4B211C1B6810203D
:101F00001A7905336270A270DB7FBA69E370637976
:101F1000B3431D43657100920022131C05F0C6F9FE
:101F200005F0BEF83C69A04200D16CE7BD4621B087
:101F3000F0BDC046C00300207001002010B5041C95
:101F400005F016F905F0ACF8A042FBD010BD00007A
:101F5000F0B58BB000AFB86105F01CFB5F4C6E466E
:101F600023689D68DB687D625A00111C0E319B005E
:101F7000C9080E33C900DB08DB00761AB546F61A2D
:101F80006D4668460021B5467D61FE6007F064FC41
:101F90000220002103F070FD03F0B6FA01200021B9
:101FA00003F06AFD7E6A4E4A20681568B20052420C
:101FB0000368BA60321C5A439100F961B107711A83
:101FC00079609107891A3A62013B23D344683E6ADB
:101FD0003219261C5E437618B400FE68920034194C
:101FE0003C61FC69A2420BD03C690426A418A446BB
:101FF0006C697642A458B44466463460043AF0E70B
:10200000BE683A6AA419FC617C6A7E68121B3A6257
:102010008919D9E7BC690B2C5CD10220002103F09F
:102020002BFD03F071FA0120002103F025FD2B4B5D
:1020300019682B4B08681C687B6AB86143439A0097
:102040003A629A07D21A3A61FB61844666464A6848
:10205000013EB4462ED365465543FE692148B31868
:10206000121852197E6938695200B2182D18FE688C
:10207000AD0075199B003D603E6AB3420ED03D68CD
:10208000E818656904380668E858301A0025565F74
:10209000864200DA1080043B023AEDE7BD6876190B
:1020A0003E627D6AFE69761BFE617D683E69761937
:1020B0003E61CBE70C49B8697E23D2B25B4208701F
:1020C0004A708A70CB70012052237A690B7105F037
:1020D000EFF8A2E7BD460BB0F0BDC046C00300203C
:1020E00070010020FFFFFF7FC404002010B5041C16
:1020F00005F03EF8201CFFF72BFF04F0D1FFA042B3
:10210000F8D010BD01207047F0B5354A007913684A
:102110008BB0B02103904900595C324ED833324F16
:10212000012902D13268023201E03A6844321A6071
:1021300003F02AFB2D496A461732012310704B70B9
:10214000CB700020B1230B7105F0B2F8284B06A824
:102150001B680024393319784900013105F0C1F9B1
:102160003A686B46DD7D13199B7CFF225BB2ED184C
:102170001C4B1B685B79D31A9D420DDD32680895B4
:102180005379FF22D31A1B4909930020D22308AAAE
:102190000B7105F08DF8F1E7114BEAB21B68069858
:1021A0000293039B07990093E3B20193002300F08D
:1021B000CDF9029A13193933FF3301345871032CC6
:1021C000CED1074A13689E2252009A5C9B1839337D
:1021D000FF33587905F0C6F802200BB0F0BDC046B9
:1021E000700100203C09002038090020EF01002088
:1021F0005C090020E801002008B503680079012887
:1022000004D11968FFF77AFB032004E00238434247
:1022100043410520C01A08BD037A70B506784568A9
:10222000012B05D0022B05D103F01AFD002302E09B
:10223000042401E001230524044A70B21268291C19
:102240009269FEF77DFC201C70BDC0467001002025
:10225000F0B593B002AF06680479057B07F08EFAFB
:10226000786205F0A3F978610520F860022D16D197
:1022700003F0F6FC7D69002360B229783268009390
:10228000F861FEF721FC884BF8691D689E235B000E
:10229000E95C03F059FDFC3568640325FD60834B60
:1022A000381C1B682C30393319780025490001315E
:1022B00005F017F9EAB2F86A396B013505F088F9CB
:1022C000032DF7D17D6964B229787D6AFC6132689B
:1022D000002D3FD100957B6AF869FEF7F5FB744B42
:1022E00074491B68386218681B797F224B708B70A9
:1022F000CB780225934380222B4352421343CB7069
:10230000602308700B713268042004F0D1FF6A4D1D
:10231000386A2C68E08107F03BFA386207F034FA3B
:10232000211C031C201C3A6A0E30103105F00CFCF5
:1023300062497F20CB7802224A70834302221343F2
:102340002A680340CB700E32F223786A0B7104F0D6
:10235000AFFF07E0584B1B681B8A0093F869002306
:10236000FEF7B2FB00237B634F4B01241B68FC3359
:10237000DD6E1B6FBD63FB636D46BD614C4D6846F2
:102380002B687A69DB685B000833DB08DB00C01A66
:10239000854602A939621178474AE3B210687A6A21
:1023A000043252008218D28800923A6AF869FEF725
:1023B0008BFB2A68A500D368AC463B6100233969D2
:1023C0008B4210DA381C6546343028583D6A590073
:1023D0006D5A78603068BD60455AB8680133451B56
:1023E00078684552EBE71368324904200B70137983
:1023F0003A6A4B708B707E235B42CB7060230B710B
:1024000004F056FFBD690134AD46032CB4D1264D0E
:102410009E2328685B00C35C002B06D0244A3168E9
:102420001268D068002205F04FFA2C689E235B00EA
:10243000E15CF86903F088FC1D4EFC34336860648D
:1024400019681C4C1B797F226370A370E37821709C
:10245000934302208021034349420B43E370F1235D
:1024600023712B68211CFC33DA6E002004F020FF5E
:1024700033687F201A681B7922706370A370E37839
:102480000221834380220B4352421343E370F22321
:1024900023712B680020FC331A6F211C04F008FF05
:1024A000F868BD4611B0F0BD700100205C09002045
:1024B000C0030020C4040020C4030020EF0100205A
:1024C000F0B5174B87B01A68B0235B00D25C0C1CC8
:1024D000076846688568C368012A05D1F8B2311CCF
:1024E0002A1C00F08BFB16E05A78197812020A4376
:1024F0009978FFB209040A43D9786846090611435E
:1025000005910B22191D07F065F9381C311C2A1C96
:10251000059B00F0E5FD2070207807B0F0BDC046B7
:1025200070010020F0B50024251C85420CDA0E59FC
:102530001759BE4200D216510E591F59BE4200D93A
:102540001E5101350434F0E7F0BD0000F0B595B040
:1025500000AFFB62C94B38641B6879645B796C20FF
:102560005900D21A0131C65DF9633A62C4490025A7
:102570003A1CBA23281C48320B71BE64FD6404F077
:1025800097FEF86B6C467C634400231C0833DB0821
:102590006946DB00C91A8D466A46386A6B002918FD
:1025A000D152F96B01358D42F7DBCDB2B54902232B
:1025B000CB70002063234D700B713D6304F078FEF7
:1025C000231C7D6B0833AD46DB08DB006846C01A70
:1025D0008546C01A6D4678628546C01A8546FD61FB
:1025E0000021221C6D467D6307F036F90021221C74
:1025F000786A07F031F9311C072002F09FFFFE6A6C
:10260000012E12D0A04BA0221B68D20538331878B7
:10261000546980069D49C00EC002214001435161AA
:10262000381C1978403004F05CFFFC6B6401BC611D
:10263000BB696E460A33DB08DB00F01A8546C01A18
:102640006C4685463E60201C0021BA696E467C615E
:102650003E6107F001F93869FF21BA6907F0FCF81B
:102660000024864BBC631B68BD6B1B799D4231DA2D
:102670003D6A0024EDB2281C7D6003F092F803F05F
:1026800063F802F051FF3E697D69BE62F86B013468
:10269000E617C30F84425E41F6B2002E06D1796878
:1026A0000819C0B203F07DF803F04EF803F00EFAFB
:1026B000BA6A011C2B1C0820FFF734FFBA6A2035C8
:1026C0002032BA62002E02D102F02EFFDEE7BC6B90
:1026D0000134C6E700247E693D696301F118E818FA
:1026E00000231A1CCE58C5580433761BB4466244E6
:1026F000202BF7D13B1CBA64386C4833796C01222B
:1027000003F0DEFBB86CFE69FD6B63000134F05230
:10271000AC42E0DB7A6B5E480023FE695900715AD7
:10272000884204DD3C6A081C1C19FC60BB601488EC
:102730008C4200D21180FD6B01330232AB42ECDBE4
:10274000FEF762F9FE6A012E5AD1BC687D6A630009
:102750007C6B5E531B5B0025BB632B1C7E6A5A009F
:10276000B15A002906D07C6BA15A0A1CA94200D29A
:102770002A1C95B2FE6B0133B342EFDB414C3E6B3A
:10278000B8236670211C022600207A6A2371E67045
:1027900004F08EFD386BB9236070211C7A6B002029
:1027A0002371E67004F084FDFB6B6C460733DB0895
:1027B000DB00E11A8D466A4600237E6B5900705A91
:1027C000FF210009FE2800D8C1B2FE6BD1540133AD
:1027D000B342F2DB2B493E6B0123CB700020BD23BB
:1027E0000B714E7004F064FD2549A5463A1CBC6B84
:1027F000B72300204832BC64FD640B7104F058FD1F
:10280000204900243D6B0223201CFA694D70CB70D7
:102810000C7104F04DFDBE681949FD683A1CB223E5
:10282000201C4832BE640B71FD6404F041FD04F0CD
:1028300037FC3E68FC6AB546002C0ED1124B1F22B5
:102840001B6839331978A023DB05114058690F4AFA
:10285000C90202400A435A6107E00638C0B20128A3
:1028600000D8E5E6FD6A012DE8D1FE68F4B2201C2F
:1028700002F097FF201CBD4615B0F0BD3C090020BA
:10288000E8010020EF0100205C090020FF07FFFFA6
:10289000FFFFFF7FF8B5141C061C06F06FFF051C38
:1028A00004F006FC071C04F019FC032C02D0002FD6
:1028B00003D107E00124002F27D0002004F000FC02
:1028C000012422E0012C03D0022C04D1381C00E0AA
:1028D000201C04F035FD04F02DFD2D4F041C3B6839
:1028E000D4331B7883420FD0002802D01123012556
:1028F00001E01223051C27490020021C0B7104F083
:10290000D7FC3B68D4331C70052406F037FFA8427F
:1029100032D006F033FF06F061FE281C06F05EFEA2
:1029200006F02CFF281C06F023FF06F0F5FE012C14
:102930001FD0174F9E253B686D005A5D002A09D0B5
:10294000154B311C1B68D8680023FEF795FC3B68CB
:1029500000225A5504F036FE0220002103F08CF8C4
:1029600002F0D2FD0120002103F086F8FEF74CF8BA
:1029700002E0002003F008F904F0C0FB051C05F09C
:10298000D7FA0379AB4200D00571201CF8BDC046D0
:1029900070010020CB040020C0030020F0B5714D71
:1029A00099B00468286802AF39602C2200213030C9
:1029B00006F052FF381C00212022183006F04CFF90
:1029C0006948036802205A6819687A769A683976E5
:1029D000BA760533DB7F7F21FB767B7F01328B4329
:1029E00004210B437B772B6892005B69391C9A1892
:1029F00000920022131C183104F058FC5A49684612
:102A00000B6838611E689B68B21C5B005A43111C3E
:102A10000831C908C900401A854602AD5B0800218B
:102A2000281C7B6106F018FF7B6901365E43013686
:102A30007600AE1961682068E2682B1C0096FEF7EC
:102A400087F9F8603869F968854605297FD14648D5
:102A50006B4606687B60F16A68460A01131C0833FE
:102A6000C01A854602AD0021281C06F0F5FEF26A68
:102A7000281C2169FEF770FA3B4968460B68002163
:102A80009A6A0E235A43131C0833DB08DB00C01A72
:102A9000854602AE301C06F0DFFE6369281C311C3F
:102AA0002269FEF795FA314B1B78002B03D121697F
:102AB000301C00F053FE06F081FC83000733DB0876
:102AC000DB006946C91A284B8D461C6802AAA36A16
:102AD000BA607B610E22013B5343F618051C043695
:102AE00038617B69013B7B610FD30020335E002B93
:102AF00009DD3969BA680139880039611018311D5A
:102B0000042206F067FE0E3EEBE73E1C383600213D
:102B10002022301C06F0A0FE61682068A368717056
:102B200010493070B37009680534E27FC96A013317
:102B3000F2705B007E22CB18524272710093EAB2AF
:102B40000320311CBB6804F0B1FB7A68954602F0A3
:102B500061FE02F085FFF8683B68BD46187017B04B
:102B6000F0BDC04670010020C0030020A005002079
:102B7000F0B59BB01C1C051C079004206E460E90FF
:102B8000A0680022012302270736139732700293B0
:102B90000392049205920693089209920A940B9369
:102BA0000C920D920F90109311921294149315930E
:102BB0001695179118941990171CB90002AB3F0194
:102BC000D8190C4BCB58311C98470B4B071C1A6873
:102BD000B1235B00D15C012902D10021D15403E073
:102BE00004F05EFAA842E8D02069FEF736FA1BB07E
:102BF000F0BDC046C401002070010020F0B5D74DE3
:102C000097B000AF161C7B6160222B680024FF3256
:102C10001C719C541C613861B96005F08FF9D04B70
:102C2000D04A796912681B68FC633C647C64F9646F
:102C30003C657C65BE63BE64DB8E5078FA215843E8
:102C40008900FDF717FD2C68AE23BA685B00E052DF
:102C5000396913788B4204D004F08AFA3B69BA6868
:102C600013702B6800229A60BF4A1278002A03D1A1
:102C7000BE4A1278002A06D0AC3301221A7030689E
:102C8000F168FFF707FE04F067FBB44C9E21236850
:102C900049005A5C9B183933FF335A79824201D07C
:102CA000587180E1B24AA62300201371111C021C46
:102CB00004F0FEFA78693168FEF7E4F923683821F8
:102CC0001879C9198200AB4B00010818391CD35878
:102CD0001B31984722689E214900535CA64DBB6278
:102CE0003A1C0023FB620C20E723291C28322B719D
:102CF00004F0DEFA9C4B1B78BB60002B00D092E006
:102D00009A4B19786B46FB60002900D0C5E0381C4F
:102D10001022283006F0A0FD21689E225200885C17
:102D20003B1C391C3A1C1C3228331E3103F010F9AD
:102D3000391C0820283104F06BFD23689E214900CE
:102D4000585C03F091F81C22BB5E3A1C291CB86049
:102D50003B627862E8230C2020322B7104F0A8FA41
:102D6000BA681E217B5E7A623A1C3B620C20E92322
:102D7000291C20322B7104F09BFA21681C23FA5E77
:102D8000081CC030C231BB68FDF758FE2368291CFF
:102D90001A1CC0321288C2333A621B883A1C203295
:102DA0007B620C20F1232B7104F082FAFEF7E6FA25
:102DB00004F0B2FA714C2070002801D004F0B2FA8D
:102DC0001E217A5E654B182A02DC2278002A08D080
:102DD0001A68111CD4310978002902D1AC320121C2
:102DE00011701B68AC229A563068F168FFF752FDEB
:102DF000051C1E22B85E624B182802DC2278002ACD
:102E00000BD01A780132D2B251B2012905DD00226D
:102E100031681A70FEF780FD00E01A70052D00D1B0
:102E200091E0FD768FE0236864219868FDF778FCD7
:102E30000A1E05D14E49D52316200B7104F038FA2D
:102E4000464B1A68136CD26B5B42934200DA131C38
:102E50003B840024381C00211022283006F0FCFCA2
:102E6000391C3A1C3B1CE0B21E311C32283303F0E3
:102E70006FF80134F98B3A1C203263009952032C0D
:102E8000E8D1404904234B707E235B42CB7016206F
:102E9000EC230B7104F00CFA57E004F057FA786059
:102EA000381CB9681022283006F0D6FC21689E2212
:102EB0005200885C3B1C391C3A1C1E311C322833E2
:102EC00003F046F821689E2252008B5C3A1C3B625C
:102ED0001E217B5E20327B62291CFF23B8682B7188
:102EE00004F0E6F923689E2149005A5C7B689A4207
:102EF0001ED0254B31681B68D8687B68FEF7BCF98B
:102F00000220796802F0B8FD21689E2252008B5C95
:102F10003A1C3B627B68291C7B622032E623B8683E
:102F20002B7104F0C5F923687A689E2149005A5430
:102F30000A4BAC221B6830689A56F168FFF7AAFC6E
:102F4000052800D0F876FB689D46104B1A68104B98
:102F50009A421FD002F00EFFFEE7C046700100202B
:102F6000380900203C090020A0050020A805002009
:102F7000CB040020DC010020E8010020E803002051
:102F8000E9030020EF010020C00300208C0900208D
:102F9000CDCDCDCD274B284A1B689968914202D0F0
:102FA0009A6801329A60254C2068FDF7DBFA2368A5
:102FB000002813D1002B09D172B6214B04211A78B5
:102FC0000A431A7080230222DB05FAE7BFF34F8F12
:102FD0001C4A1D4B1A60BFF34F8FFEE7013323607D
:102FE00023682F2B01DD00232360FB7E114C052B72
:102FF0000CD004F06BF82368B02252009A5C824235
:1030000013D00121B1228A4099540EE004F05EF8F9
:10301000B02321685B00CB5C8342EAD104F040F826
:103020003A69904200D12EE6E3E7F87EBD4617B03C
:10303000F0BDC04670010020FFFFFF7FA405002007
:10304000290000500400FA050CED00E0F0B501275E
:103050009FB00A97052712979F6800240222051C3B
:103060006E4602A81B911B490736069207900E93E5
:103070000F92139714921693062719921C931D9082
:103080003F23201C221C3470089409940B950C9447
:103090000D94109411941594179718941A950B7118
:1030A00004F006F9A20006AB240118190A4B311CE2
:1030B000D3589847041C04F009F8084B1A68B02349
:1030C0005B00D35C834203D103F0EAFFA842E9D05E
:1030D0001FB0F0BDCB040020C4010020700100200F
:1030E00082B00020019302B070477047F0B5A1B0E4
:1030F00000AF786301F05AFFB86101F045FFCA4B99
:1031000078611C686846636822685D005A43FD6107
:103110005500D2185200131C0833DB08DB00C01A1C
:103120008546FD6000216D463D6306F095FB6368B2
:1031300022689E005A43D3189A00131C0A33DB08F6
:10314000DB00E81A85466D4600217D6206F084FBAF
:10315000636822689D005A43D3189A00131C0A33EF
:10316000DB08DB006846C01A85466C46FF21BC625E
:1031700006F072FB7C6B013C3C620024FC623C6A02
:10318000162C19D80124386A231CA84A83401342FC
:103190000DD1A74A134206D159050DD5201C03F0C5
:1031A000E1FFFC6208E0A34B1B68303302E0A14B57
:1031B0001B6832331B78FB62FC69B6083E61640809
:1031C000AD08FE6AFC61BD60013E701C00D1A3E049
:1031D0003D6A022D06D97C6B0B2C03D0231C113BBE
:1031E000012BF1D80220002102F046FC02F08CF9FC
:1031F0000120002102F040FC8B4B1B681B68FB6325
:10320000FB6B5A1EFA63002BDED0874B1B685B6892
:103210003B643A6C531E3B64002AF1D08248864AD4
:1032200004681168FA6BA468501C604318180130D8
:103230004D697C6B80004059032C43D004DC012C89
:103240000AD0022C17D0E4E77D6B0B2D28D0E0DBF1
:103250002C1C113C012CDCD8BD69EC183834A57845
:10326000CC697969AD00373109782C59CC40001B05
:10327000C143C917084039697C6A5143591889000C
:103280000C597D6A00194851002EC2D1FC69F96AB7
:1032900062439B185C00FDF79FF93D6B6053B8E7F4
:1032A000BC69CA69E31838339B7899007B698A58EE
:1032B00037331B78DA40801A3128AADC002003F06B
:1032C00051FFA6E73C69544319198D00796A6D587E
:1032D000011EA94200D2291C7D6A1C19A40061515B
:1032E000BC6854431D19A446BC6AAD002D59A842C0
:1032F00000D9281C65465C19BD6AA4006051081AF3
:103300007F24FD2801D8400884B2FD696A433D6BE3
:103310009B185B005C537CE7434E381C33680021EC
:103320001C685D683C62FD621C690533DB7F1A2204
:103330004430BB6106F090FAF968386B7A6B451837
:10334000291C00F06DF97A6B112A77DB122A0BDD4C
:10335000132A73D1291C386B002202F0DBFFFD6AAF
:103360007D630025BD616BE07C6B112C0CD1336853
:10337000FD6A5B68013D7D63013B00253C1CFD60EF
:10338000BB60403401250DE033683C6AFD6A1B6870
:10339000013C3C62013B7D633C1C0125FD60BB6040
:1033A0003C3400257D6135682868F863FB6B591E45
:1033B000B962F963002B34D0696839643A6C531EE2
:1033C0003B64002AF2D0B86AF968FE69421838698D
:1033D00042437869C1188A18796A92005058B96ACC
:1033E0003A694E434A4384469A18786A92001258C2
:1033F0002168B8689E19760081420EDA6146FA208B
:103400008B1A8000891858434910002900DC0121DB
:10341000FDF730F93A6BB052D0E7386B00233352E6
:10342000CCE71C1C0CE0C046C00300200400400098
:10343000030003003809002070010020FD6A7D634D
:10344000386A796BBB693D1C6035FA6A287069700F
:10345000EB70381C391C7E235B42AA7044311A225F
:1034600066306B712C7106F0B5F9281C396B03F0CE
:1034700091FEBD4621B0F0BDF0B5504C87B0066856
:10348000406800AF2568AE23BE6078605B0039609D
:10349000E95A2869FDF744F9494B39611B68986975
:1034A0005A69410001324A43131C0833DB08DB0030
:1034B0006946C91A8D466E46301C00217E6106F0B1
:1034C000CBF9A9697A68786904F0B4FBF86004F074
:1034D00079F82368AF223B4D5200002199542968A6
:1034E00094468E6B4268B24203DBCE6B81688E429B
:1034F00005DA181C01217E30017060461954F96804
:103500006026FF3601290FD19955081C01F09EFF56
:1035100002F09AF902F0B6FA22689E235B00D15CB1
:10352000022002F0BBFA3EE060461B5C002B06D195
:10353000254B78681B6879695A7804F083FC216808
:1035400000238B5502F080F902F09CFA2A68236868
:10355000AE21343249001278595A3E69891AB14273
:1035600001DD964220DC196991421DDD3E69002E85
:1035700008D101F0C9FF20689E235B00C15C0220D6
:1035800002F07AFA2B683E6934331B789E420ED1E2
:1035900023681A1C7E321278002A04D1BE685A6948
:1035A00003CE04F039FA23687E3300221A703E6895
:1035B0000523BD46337007B0F0BDC0467001002042
:1035C000C0030020380900203C09002008B503F0A2
:1035D0008BFC08BD104B10B51B681A6B002A03DD6D
:1035E000996B5218D10F13E000218A4210D10B4978
:1035F000986B09680624095F9E2464001C5D002CFA
:1036000001D0C82252428A180121904200DB0021D9
:103610006833197010BDC046700100203C090020BD
:103620007047000008B502F077FA01F01DFE01F0C6
:10363000B3FD01F067FD0F4B1B681A7A0E4B1B6838
:10364000D433002A01D0022200E003220B491A6081
:1036500000230B700A49A0220B700A49D2050B7097
:103660009363D36B3F218B43D36362B602F0E4FED6
:1036700008BDC04660090020E40100202900005078
:10368000280000502A00005038B5051CFDF722F92B
:10369000041C04F033FCA4235B00E35C002B28D063
:1036A000144B00221B68DB6A013B07D31901691820
:1036B0000820095E0029F7D10122F5E70E4B1968B1
:1036C000086B0B1CFC33002811D1896B00290ED12B
:1036D000002A0DD01A6DFE2A01DC01321A651A6D1E
:1036E000052A06DDA42100224900625400E00022E0
:1036F0001A6538BDC00300207001002070B5051C9C
:103700000C1C161C03F06EFD002802D001280AD004
:1037100023E00E204643AD19EA88FF23FE2A00D895
:10372000D3B2637119E00E2070432818C288FF23BA
:10373000FE2A00D8D3B263710B220A238256C356E5
:103740000921D31A0822415682568A1A934202DD71
:10375000A371E27101E0A271E37170BDF0B58DB0AB
:1037600005900C1C012603F043FD059D0296634B5A
:10377000029E1B68013E1B6A01969E4200DBB1E07F
:10378000238808AE33806388301C738005F0A8FD61
:103790000427EB5F002B76DD2B8807AF3B806B881F
:1037A000381C7B8005F09CFD3888338803907F8827
:1037B00004970221705E3FB2381AC2178018504039
:1037C0004F4A019E1268BC469219283211784D4A20
:1037D0001268002901D1453200E046320427E65F35
:1037E000039F127839B2002E08DD904206DA1BB230
:1037F000CB1AD8171B184340934269DB09AE3378C4
:1038000080277F421F43DF200740287B012340227F
:103810001840174310239F430001029A0F23384397
:1038200098431A4002433270727809129A43194041
:103830006746114338120B4000011843AA88707084
:1038400004990398131C12B2B070F170FF2A00DDC6
:10385000FF23019A0598311C3371FFF74FFF301C8D
:1038600003F0D0FC0423E25E254B1B68002A04DD34
:10387000019E01229B19283303E0019F0022DB19DE
:1038800028331A7020E00420235E002B20DD09AFCE
:1038900000210C22381C05F0DFFF029A0F231A408A
:1038A00040210A433A700122B25603203056944612
:1038B000318872886646000133400343381C7B70B0
:1038C000B970FA7003F09EFC2B8823806B886380AC
:1038D000AB88029FA380EB880137E38002970E3507
:1038E000083444E7064B1B681A6C191C34310A7003
:1038F0005A6403F09BFC0DB0F0BDC046C00300202D
:10390000C803002078090020F0B5D44B9BB01B6899
:1039100000250593D24B0D901B6810911E6A0E2353
:103920007343C4180C9311960A94231C321C0695F9
:103930000B950E3B013A0BD3D988069F8F4200DAD4
:1039400006910420195E0B9C8C42F2DA0B91F0E791
:10395000C44C012123681A1C5232127891401A1C5F
:10396000533212785433891A1A788B1ADBB21393B4
:10397000FCF7B0FF23680F901A1C383212780E92B1
:10398000B0225200825C022A03D1B74B1B68E1339C
:1039900006E062220F9DFF32AA5C022A02D139336F
:1039A0001B780E930C9B0D9C0E3BE318771E1C1C82
:1039B00008970793059D331C82270933BF009B009E
:1039C000EA19D31804340993013E00D2F2E0231F10
:1039D0000020195E0E9D0023E25EA44B02959942E1
:1039E00004DC01270297002A00DC02959D4B029D12
:1039F0001B68191C38310978A94213D1059F822010
:103A0000800039188919097D49B2A9420AD1109D4F
:103A1000F10069180427C95F002903D0191C393146
:103A200009780291002A00D1BFE01A1C47321578AC
:103A30000F9FB0225200BA5C012A04D11A1C608880
:103A400002CA14330AE0022A0BD1874B60881B6834
:103A50001A1CF8320D331168FF33043203F064FD91
:103A60000390A4230F9F5B00FA5C7E4B002A06D0D4
:103A70001A68039F29321278974200DA03921A6873
:103A8000131C48331B78002B01D164234CE02B1C02
:103A9000774F059DEF191497787B1590002822D158
:103AA0000021675E64217943C12080008C4629187B
:103AB000039D5D43AC4514DD039DAF4211DC8F686F
:103AC000BC460127BC44684F60463F6888606C373D
:103AD0003F78BC4507D1149D01276F73159F8F60F8
:103AE00001E000208860059F61483D18697B00293E
:103AF00014D00027E15FC120059F80008C46391853
:103B0000039FBC4508DD8868029F01308860B84289
:103B100004D10020687300E000208860059D544FA8
:103B2000E919497B0029B0D0059D8227BF00E9191A
:103B30008819057D0027E05F002D03D0029F6DB23C
:103B4000BD4221DC039D642141436B4399420EDB5E
:103B5000131C44331B78069F61887B439B11994259
:103B600005DB136C0B9D6B439B1198421DDA099F7B
:103B7000002363802380059D3B608227BF00EB19F3
:103B80005A68013A5A6010E03A4D28326843127878
:103B9000039D6A435343984207DA099F00236380D9
:103BA00023803B604B68013B4B60099D0E3C043D0C
:103BB000099509E7059E8227BF00089CF31900229A
:103BC0005A60119D1A19109E14320D9F0C9C06927A
:103BD000EA00B21803923A190C3A0292089A089D28
:103BE0006C3252009A1804320C92089A822674326F
:103BF00052009B1808330D930C236B43B600059FAE
:103C00009B19FB181093089F013700D1C0E2079D54
:103C10000A9C0E9E0022AA5E144B0E3C0494099648
:103C20009A4208DC0A9B01240A3B0027DB5F0994C7
:103C3000002B00DC09960A9D0A3D0026AB5F0B9520
:103C4000002B00D127E2069F099A3B780632013308
:103C5000DBB259B291420FDC3B7011E0C803002087
:103C6000C0030020780900207C090020FF0100002B
:103C70000703000010270000099B069C04332370F3
:103C8000069D0023EB56012B09D1079E039B32882A
:103C9000083B029F1A80039B3A88063B1A80069CC9
:103CA00000256557012D65DDA81C0321FCF738FDB3
:103CB000039CCEB21296083C022D45D1DA4B039DEF
:103CC0001868DA4B063D196803680027E25F9C46D6
:103CD0000026AB5F4E69096940684910511ACF1739
:103CE0000138C91900027940401A7F280ADD761090
:103CF0009E1BF0176746013F36183F024640BF1B28
:103D00007F2F11DC079E029F0020305E0021795E2C
:103D1000801AC91A04F0F8FC0B2805D92388079CDF
:103D200023802B88029D2B800323013B1CD3109FF3
:103D3000079E5A00BA183088111C5A31029C08801C
:103D4000218860321180F0E7089D06236B43059EB1
:103D5000C9182288B64B49007118CA52039B063B0A
:103D60001A889A239B00CA52079F029C3F88248886
:103D700019971894AF4B1B681A1C883211780129C7
:103D80001ED189331B78089D9D4219DA0F9BD433CD
:103D90001B78002B14D1D4216943A44B069E1B68C9
:103DA000603159180023F3560092A34A0498126810
:103DB000383212780192039A083A00F033FD52E14A
:103DC000069F0026BE57012E00DC4CE1079C002513
:103DD000655F032E00DC33E1089C062767431298D9
:103DE0000599C4196400924A0C19A25A043003219F
:103DF0001192FCF795FCCAB2059BD21952009A1891
:103E00008B489A239B00115AE05AD35A14909C462F
:103E1000042E0FD1039B083B0022985E281AC3177B
:103E2000C0185840039B029D063B0022AA5E002654
:103E30009B5F0CE00C9E0020305E0D9E281AC2177E
:103E4000029D801850400023F35E0022AA5ED31A20
:103E5000DA179B18059D089E5340784AC018AB1985
:103E60009B181D78744A002D06D015685A352D8888
:103E7000A84208DC002505E015685C352D88A842BD
:103E800001DB01251D701B78002B31D112688021C8
:103E9000131C5832128856331B8800924A0003F0D4
:103EA00032FB634F079D061C0021695EE05F029FA5
:103EB0000B1ADD175A196A4000257D5F9A27BF004B
:103EC0009446E25FAD1AEA17AD18554065442B1CC5
:103ED000321C05F07DFA079B321C1880E05F029CC3
:103EE0002B1C0021615E05F073FA029D288077E0AB
:103EF000119E149DB4B2611A09B26646AAB2CB0FE4
:103F00005918931B1BB2DD0FEB18079D5B100026A1
:103F1000AD5F49100495029D16930026AD5F6318AE
:103F2000169E049C17951BB2E31A9219179CDD1775
:103F300012B2A21A5B196B40D51752196A409B182E
:103F400015910024802B01DD1C1C803C129803215C
:103F50000530FCF7E5FB384BC9191F68119A059E1F
:103F60003B1C533349005D78711810B21E78304AFB
:103F7000139B58438B5E7343C018049B6B43C0185C
:103F80003B1C52331A7855371041119014983B78E6
:103F900007B2139847439A208000095E4E43BE192A
:103FA000179F16997D437519159E59437343119FA9
:103FB0001141134115418022F8186D18231C0499F2
:103FC000D20005F005FA079E029F30808022231C54
:103FD0000021795E281CD20005F0FAF9029C2080AD
:103FE000039B0B9E043B0021715E0025585F124D20
:103FF000431A2F68DC171B1963403C22BA5E05F098
:10400000E7F90B9E039B0A9C3080023B083C188812
:1040100021882B683C27DA5F431ADD175B196B4058
:1040200005F0D6F920801EE0C0030020C803002060
:10403000620200007C09002078090020DA020000FA
:10404000039B079F083B00269B5F029CED18039B88
:104050006D103D80063B0022A25E00255B5F029E44
:10406000D3185B103380069F0022BA56099CA242E7
:104070006CDD0B9D0023EB5E002B74DD039B043B8A
:1040800000269B5F002B6EDD199C0C9F189E0D9DDA
:104090003C802E8067E0069C0022A256099DAA4221
:1040A00030DD0399043900268A5F002A32D0059F4B
:1040B00082208000089D3A185419A07F0130C0B2B8
:1040C000A077344C40B224683A342478A04202DD10
:1040D000069E33701EE0039B079F083B1B88029CD3
:1040E0003B80039B0B9D063B1B8823800B882B800A
:1040F000039B023B19880A9B083B198053680133D4
:10410000536007E0059F089C234D069E3A195219FB
:1041100033701370089E069F013E039C079D08960E
:104120000A9E013F083C0E3D0E3E06970394029FF7
:104130000C9C07950A960D9D109E0E3F023C023D79
:104140000C3E02970C940D9510965CE501230B9C98
:104150005B422380059D8226B600089FAB19DB19C0
:1041600000229A77D6E7059D8226B600AB195968DA
:1041700001315960074B1B6838331B789A4201DACA
:10418000069F3B7062230F9C0022FF33E254E1E75D
:104190001BB0F0BD78090020DA02000008B5FFF777
:1041A000B3FB08BDF0B58FB0059007910A920B9351
:1041B0000024404B1B68DB6A9C4278DA059F230190
:1041C000FB1808201B5E002B6FD0079FA300FB1875
:1041D0000327DF5708979B78013F5BB2069304974C
:1041E000089F049801370997B8425EDC069E013E9D
:1041F000069B01339E4255DC2E4B04991B6801310E
:104200009A680A9F5143481C80193D5C013D47D381
:10421000DB6A9D4244DAAC4242D0079FA300DB5FD9
:10422000254F40003F687F8EBC46149FC05B834291
:1042300036DC069F6046C91943430131149F49008B
:10424000C95B9B118B422BDA099F7A43B21801326A
:10425000149F5200D25B934222DAA54202DB2B1C50
:10426000251C1C1C059821010DAF41180A31381C72
:10427000042205F0AFFA059A29015118381C0A31B9
:1042800003F0C8FE00970A9F231C01970B9F059817
:104290000297149F079903972A1C03F0D9FE2C1C40
:1042A0000236A5E7049F023799E7013481E70FB092
:1042B000F0BDC046C003002078090020F0B593B0DF
:1042C0000A9210900C1C05F059FAAA4B11901B6829
:1042D00007259A7A0795062A00D80792A64A1168F8
:1042E000A42252008A5C002A05D19E7906960820F5
:1042F0001F5E059706E0A14B1B681D7A06950A27ED
:10430000DE5F05969E4D9F492B680A9F5A68186884
:104310004A709A6804238A70013292000870CB7048
:10432000BA18512302200B7102F0C2FF0022A31D14
:10433000DA770233DA777F26631DDE772968E31D9B
:10434000DE7748680B680138C0B20C908A48013BA0
:1043500005685BB2281C7A30028042808748AC46F0
:10436000006803920D908848029200680E9087487A
:10437000006808907F4800680490002B00DAC0E0D5
:104380000C9E5F0072B20997002A00DAB7E08D68D0
:10439000581C6843013080180A9E0D9F00908500CC
:1043A000AD593E7B002E27D0119E0E980436760024
:1043B0008619F68867467543B0267600BE5D9E274F
:1043C000019601986A26ED137F00FF36022808D176
:1043D0006046C75D08987E430F68C018574386192A
:1043E00007E06046C75D08987E434F6886195F43C3
:1043F000D719F65D7543AD114E68189F5E43961947
:104400007600F65F109F751B009E7000C553002D4F
:104410005BDB042D04DD60467A30068801360680B9
:10442000049E0C203056854213DB2768281A381862
:10443000206060690D2701306061F757301C0C2641
:1044400086576068BD4201DCAE1B00E0BE1B8619CA
:104450006660E668B54204DDD7B2DEB20F970B9610
:10446000E560079FBD421BDB201C08301F268657D6
:10447000964200DAC277E01D1F268657964200DD7D
:10448000C277A01D1F2686579E4200DAC377601DA3
:104490001F2686579E4200DDC377039E0136039692
:1044A000AFB200971A9F5600B85B009F38181A9F4A
:1044B000B853199E0998375A009EF019199F099E02
:1044C000B853029F7F19029717E060467C30068838
:1044D00001360680049E0E203056854206DCA76811
:1044E000281A3818A060A0690130A06120698542AF
:1044F00000DA2561029E761B0296013A44E7013BF1
:104500003BE71F4B02981B680125D968FCF7B2F8FE
:104510001F497C235B42221CCB70E06176231C3256
:10452000281C0B714D7002F0C3FE039FA21D276271
:104530001F21631D51561F229A56134B1B6891422F
:1045400001DB1D7301E000221A730F9D231C0B9EDB
:1045500028331D705E70E768069D0120AF4205DAC2
:104560002369059ED80FF2179E425041C0B213B086
:10457000F0BDC0466C0900207001002074090020C5
:10458000C0030020C4040020C403002070090020E0
:10459000EF0100200B4B09681A68B0235B00D35C65
:1045A000094A1268D07A48438011012B01D1937ACD
:1045B00004E0022B05D1054B1B68DB79984200DA39
:1045C000181C7047700100206C090020740900203D
:1045D000F0B591B00D1C1E1C0E92089002F0E6FF83
:1045E0008D4B0A901A680321177A20240597577A71
:1045F00006975156894F641A02213B685156907AAA
:104600006400641A19781B790090D27A6410E4B2BD
:10461000029401927268169804F002FF3B68059FAD
:10462000197972681B780097069F02940197179872
:1046300004F0F6FE6F7A7F230B97AF7A0024099778
:10464000EF7A2E7AAB722B726C72EC720C9702F0CE
:104650004DFD76B20F9002F059FD06940B9F7BB290
:104660009E4200DDA9E0099F73007CB2169FFB18F3
:104670000D930C9F7BB2771C07979C4200DD9AE05C
:10468000664B079F1A6893687B43E3180E9F0133BC
:104690005B00D95F179F6300FB181B890D9FC91A28
:1046A0003B890A9FCB1A0593BB7A059F9F4214DD75
:1046B0000B23EB56A34200DAEC720A23EB56A3421B
:1046C00000DDAC720923EB56B34200DA6E720823A8
:1046D000EB56B34204DD2E7202E0059F002F5BDD36
:1046E000069F0598874200DA06900F9F002F55D04D
:1046F00013685168DF17BF0FFF18BF10CA17BC46F9
:104700000497920F012752187F429210481EBC4412
:10471000801A664510DB049F0137BE420CDC531E35
:104720009C4202DB0132944260DD431E9C4235DB39
:10473000013084425CDD31E0DF0FFF187F10BC46A2
:10474000049701277F42BC4466450CDB049F013778
:10475000BE4208DCCF0F791849104F1EBC4202DB65
:1047600001318C4246DDDF17BF0F591EFB189B102D
:10477000CB1A591E8E4211DB01339E420EDC531EB2
:104780009C4202DB0132944236DD431E9C4205DB33
:104790000130844232DD01E0002705971F4B079F5F
:1047A0001B6805989B687B43E3180133089F9B00B7
:1047B000D85101345DE73E1C50E7184B18491B687F
:1047C000069F5A682F6018684A709A68089F8A7016
:1047D0007C2301325B4292000870CB70BA188323AD
:1047E00005200B7102F064FD11B0F0BD012706E059
:1047F000042704E0022702E0002700E00327FFB2BD
:10480000381C02F08FFC05998842C7DA059801B27E
:10481000381C02F095FCC1E780090020C00300208D
:10482000C4040020F0B5E5B014926AAA20CA0D9025
:104830001278281C19920A1C0491D0324830117841
:104840000078884201D301311170CE4A0D9F16685D
:104850000022BA5E306D0D9D42431214179202225F
:10486000AA5E776D7A4312141892012B39D1049AFB
:104870000021D1321170049AD0321370049B179D1D
:10488000189F002201311D60DF605A601A619A6032
:104890005A619A61DA611A625A629A62DA62343350
:1048A0000429ECD16A9B049D9A8C22332A63DA880E
:1048B0006A6659892A1C98321160D98951631A880D
:1048C000291CAA619A880431EA64AA651A89CA6710
:1048D00088310A608A609B892A1CB4321360D360D5
:1048E00053616A9D002402351A941B940395039D1D
:1048F000A20000235219181C1A255D43049FD15AA7
:104900007D192D6B023369434018082BF4D1FA212D
:104910008900FBF761FE682109196A460234885252
:10492000082CE4D11CA80021102204F095FF0025DA
:1049300034236B43049F20A8FB181B6B039F069333
:10494000EB00FB182F0107933F1800240799069AE4
:10495000085B68231B1950436A46995AFBF73CFED3
:1049600063001CAA9958F850023408189850082C73
:10497000ECD10135042DDBD1D02230A8002104F088
:104980006BFF149D376D0023EB5E149D7B431B145E
:1049900030930223EB5E726D012653431B14339355
:1049A0003DAC21AF03960023049A079306931E1C87
:1049B000181CF95815684D434019D5684D437619B0
:1049C00055684D43069949190691FD5811691033F0
:1049D0006943079D34326D180795402BE9D1039D3B
:1049E0001CAAAB009D58291CFBF744FE291C206023
:1049F000301CFBF73FFE291CE0600698FBF73AFEEF
:104A0000291C60600798FBF735FE039E2061012E8C
:104A100019D00023049A0593181CFE58916810338E
:104A200071434018516934327143059E76180596DA
:104A3000402BF2D1291CFBF71DFE291CA060059814
:104A4000FBF718FE6061039D34340135039504378C
:104A5000042DA8D138AC0025A80020A984460A1C42
:104A6000624400230992049A0A93089307930693D9
:104A70000393181C099ED769F15896694F434E431A
:104A80008019039E1033F619176A03964F43069E4A
:104A9000F619576A06964F43079EF619976A0796C6
:104AA0004F43089EF619D76A089679430A9E343216
:104AB00076180A96402BDDD167461CABFE58271CA2
:104AC000311CFBF7D7FD083F3860002D1BD0311C8F
:104AD0000398FBF7CFFD271F3860311C0798FBF7C1
:104AE000C9FD6060012D0ED0311C0698FBF7C2FD98
:104AF000311C20600898FBF7BDFD311CA0600A98AE
:104B0000FBF7B8FDE06001353434042DA4D1049BDB
:104B1000002130AA8D58521856689768D0681D60D9
:104B20005E60156956699F609769D8601D615E6116
:104B30009F61D069156A566A976AD26A3431D86122
:104B40001D625E629F62DA623433D029E1D1049C37
:104B50000026251C0835069507966A9B079F323369
:104B6000022F0BD0032F0FD0012F03D01D789A886E
:104B7000DB880CE05D781A895B8908E09D789A896A
:104B8000DB8904E0C8030020DD781A8A5B8A9C4632
:104B9000012D60D0002D4DD0022D79D1069E606888
:104BA000366827680111C9198019069F0F9020697E
:104BB0007F68089673116669CB180111C9191193A2
:104BC0007311CB181293A36A80190A96DE0F109006
:104BD000F618E06A76100596C10F266A0918491082
:104BE000F7187F180397A069E7693E18206AC70F76
:104BF0003F187F10F719E669606ABF193F180598DA
:104C00003E180398C70F3F187F10606AF719E669CE
:104C1000361805983618206A3618F018666A401853
:104C20000590F118E06AC91809181B180E9186182A
:104C3000139339E0069F26687F68A0691196129742
:104C40002E1C171813950E95039505950A9510952A
:104C500008950F9528E0666827683311DB19069FD1
:104C60000F9626697F6811933311DB19E06912935F
:104C7000A369616A4700FF18401810967F18002644
:104C8000891805900E91139603960A9608960BE0E4
:104C9000002613960E9603960596371C0A961096D4
:104CA000129608960F9611961298189B119A1B1A35
:104CB0000B93FB171B0F1799DB191B116344891A00
:104CC0000991B801191C0C93FBF7D4FC059A0C99B7
:104CD00015909001FBF7CEFC039B0C991690980160
:104CE000FBF7C8FC1199099B8A0215994B43D3180D
:104CF0009B1223600F9B16999A01099B4B43D31873
:104D00001B019B126360089B06999A01099B434310
:104D1000D3181B019B120B60129B15999A020B9BD7
:104D20004B43D318069A9B125360109B16999A0115
:104D30000B9B4B43D3181B019B1223610A9B9A01C7
:104D40000B9B4343D3181B019B126361802315996E
:104D5000DB00591A0B1C7B43DA17920DD3189B12F8
:104D60008C46A361002D05D1E56125626562A562CF
:104D7000E56234E0059B4B43DA17920DD3189B1282
:104D8000E361169B059A5F427A430E9B9902521883
:104D9000D3179B0D9A1892126262022D1BD1039DAC
:104DA00061464D43EB179B0D5D19AD122562039DC6
:104DB000B6026F43139DAB02FF18FB179B0DDF1963
:104DC000BF12A762039F7843301AC617B60D30187A
:104DD0008012E06203E000232362A362E362099A87
:104DE0000B9B52435B43D318574A934205DC642024
:104DF00058430C99FBF73EFC00E05448544B4610D6
:104E0000544D01209E421BDC301C291CFBF732FC58
:104E1000291C421C5143771AFB17FF185F404E4B69
:104E20004000C05A520078434C4FC919761AF11706
:104E300076184E40D15A4E43291C8019FBF71AFCB4
:104E400068430C99FBF716FC079F069DBE0030AB2C
:104E500001373435F050079734340695042F00D0CD
:104E60007BE60024251C68266100361930AA6F46AF
:104E7000F35B8858049E58431A236343FA21F318BE
:104E800018638900FBF7A8FB02344519082CEAD106
:104E90000024049F291C3E19306BFBF79DFB002862
:104EA00001D0306301E0012333633434D02CF0D1DE
:104EB0000024049B251C211C201C1A6B1E68013138
:104EC00056433018DE6814195643343375190429D3
:104ED000F3D1211CFBF7CEFB211C061C281CFBF781
:104EE000C9FB049D199A2B1CD033197801322C6B05
:104EF000013391420CDD1A78002A15D16A9A4632A4
:104F000095788D4210D3128894420DDB012200E087
:104F1000002200211970012A08D1149E0D9F3388A8
:104F20003B8073887B800CE001221A700C4B0D9D36
:104F30001B689F6DDB6D7E435843361400142E8032
:104F4000688065B0F0BDC04614AE4701FFFFFF7F2B
:104F50006F11010010270000AE980000F0D8FFFF8D
:104F6000C8030020014B18607047C046600900204C
:104F7000014B18687047C04660090020014B18605B
:104F80007047C0465C090020014B18687047C04656
:104F90005C090020014B18607047C046580900208A
:104FA000014B18687047C04658090020014B18682B
:104FB0007047C046E40100208D23013B002B01D047
:104FC000C046FAE7044B10221B78DBB21807C00F6B
:104FD000134018437047C0462B0000500F4BF7B5E5
:104FE00018261E700E4BA0271E70FFF7E5FFFF0569
:104FF0000B4B01AC00252C3760701D703E70FFF725
:10500000DBFF064B20703D701D7023786278181C02
:105010005040400013400343D8B2FEBD2A00005068
:105020002D00005010B50D4B00201B78AA2B12D17B
:105030000B4B1C780B4B64B218780B4B40B21978B1
:105040000A4B20181A780A4B49B21B78401880186E
:10505000C01A43425841C0B210BDC04650000200C1
:1050600051000200520002005300020054000200EE
:105070005500020030B50C4B00201A78552A11D18A
:105080001D780A4B18780A4B28181C78094B001910
:105090001978094B40181A78084B80181B78C01AE9
:1050A00043425841C0B230BD5600020057000200D2
:1050B00058000200590002005A0002005B00020082
:1050C00010B5041CFFF7D6FF002810D0092C01D121
:1050D000084B0AE00B2C01D1074B06E00C2C01D148
:1050E000064B02E00F2C02D1054B1C78E4B2201CC9
:1050F00010BDC046570002005800020059000200CF
:105100005A000200154BC0229200985814490140E1
:1051100099509958FF208143402001439950985855
:105120001049014080200004014399509858802183
:105130000002000A09060143995002221A60012266
:105140001A60082104221A601960FC33002159609A
:10515000054B19690A431A617047C04600E100E037
:10516000FF00FFFFFFFF00FF00ED00E013B5094A5D
:10517000042413780021DBB21C4301910198F4212F
:10518000FF31884205DC1370C0461470019901316B
:10519000F3E713BD0D00005013B500220192A022C9
:1051A000D205D06BC021C9000143D16301AB18788F
:1051B00003218843012108430C24A04304242043F5
:1051C0003024A043102420433F2420404024204387
:1051D000187098780F24A043072420439870D8783B
:1051E0000143D970019B936113BD00000122A023EC
:1051F000DB05104002060349986908401043986196
:105200007047C046FFFFFFFE13B51F22013001AB00
:10521000CCB2104002311870C905601C0234104035
:10522000C90D224059809200090A1143D970587063
:10523000019AA023DB05DA61196A024A0A401A6260
:1052400013BDC046FFCFFFFF0002064B000A013826
:10525000002258609A6005221A60C0461A68D1037D
:10526000FCD5704710E000E0F0B5554E85B03368CE
:10527000544F196B1A1C33331B78303215781B07C7
:10528000023212781B0F00930F231407994312095F
:105290002D0701922D0F0B1C80222B43520013432C
:1052A000494A0395494D1340494A2B404949134007
:1052B000240F0B400199220413430A054649029426
:1052C0000B40009913433B400A061343434AA02472
:1052D000E4051340E360FFF749FF3368E2683133C8
:1052E0001B781540DB069B0FDB021D43E560E2687F
:1052F00080239B001343E360E26880239B011343F8
:10530000E360029C039DFFF78DFE3E1C002813D036
:10531000334F882039781E34C9B2FBF7ABF939789E
:105320004443C9B28820FBF7A5F90F3545431E3C1D
:1053300000230F3D9C4203DB231E0F2B00DD0F23B8
:105340000F22954200DD151CA024E40521491A40D6
:10535000E36812040B401343E360EB43DB171D408B
:10536000E3680F27BB433D401D43E560E368F0223F
:10537000934380221343E360E368174A19481340BC
:10538000E360E3683340E360FFF75EFFE268802399
:105390005B051343E3600098FFF792FE0740380671
:1053A000E7683E400643E6600F48FFF74DFF019B6C
:1053B00009491A05E3680B401343E36005B0F0BDEB
:1053C0005C090020FFFFFFF0FFF9FFFFFFE7FFFF91
:1053D000FFDFFFFFFFFFF0FFFFFF0FFFFFFFFFEF0C
:1053E00054000200FF0F0000FF6F0000064A074B49
:1053F00012680120D432126819789040021C0A43C6
:10540000D2B21A707047C046E40100202900005053
:105410000549064B09681A78D4310968012088408B
:1054200082431A707047C046E401002029000050F2
:10543000044B1878044B1B68D4331B6818410123B4
:105440001840704729000050E4010020044B82B04E
:10545000019001AA188092789A7002B07047C046F5
:1054600024000050054BB2221968520000238B52D1
:10547000034A1370034B0122DA7770477001002052
:105480002009002008000050014B0122DA77704704
:1054900008000050054B1B5C002BFBD0A023DB0554
:1054A0009968034A0A409A607047C0462009002064
:1054B000FFFFF9FF72B6084B1B5C002B03D1C046FF
:1054C00030BF62B6F6E762B6A023DB059968034AEF
:1054D0000A409A607047C04620090020FFFFF9FF8C
:1054E00072B6074B1B5C002B02D1C04662B6F7E7D1
:1054F00062B6A023DB059968024A0A409A607047A9
:1055000020090020FFFFF9FFA023DB055A680121D5
:10551000120E58689143034A090602400A435A6032
:105520007047C046FFFFFFFE08B5A0230120DB0542
:105530005870FFF7AFFFFFF7E7FF08BDF7B5A026EC
:10554000041C0191F605042808D005280ED14C4B07
:105550001B681A1C883217688C3305E0484B1B689F
:105560001A1C9032176894331B6814E0454B1B6873
:105570005F6A9B6A7361FBF7ADF901F091FD022848
:105580000AD0414B01995A5C7F231A4071693F4B05
:1055900092040B4013437361A023DB051F611E6956
:1055A0001F231E40FFF73EFD00280AD0384B8820FD
:1055B00019780436C9B2FBF75DF846430023043E70
:1055C00003D4331E1F2B00DD1F23A022D205106938
:1055D0001F210B40884303431361032C1CD005DCBF
:1055E000012C21D012DC002C10D020E0052C09D099
:1055F00004DB062C14D0072C16D018E0204B1D68B5
:10560000983514E01E4B1D689B3510E0FBF762F9DE
:105610001C4B1D6835350AE01A4B1D683B3506E00A
:10562000174B1D689E3502E0164B1D683835A023C8
:10563000DB05596928783F221040914301435961A5
:1056400068781F215D6908401249C0022940014362
:1056500059611149640009680C19211C9A310878B4
:10566000596810409143014359609B342178586830
:105670000A401102094A02400A435A60F7BDC04677
:10568000600900205C090020BC030020FFFF03FE2E
:1056900054000200FF07FFFFE4010020FFC0FFFFEE
:1056A000244BF7B51A68244B1B6838331B785B060C
:1056B0009B0E0193131C3133197800238D0055196B
:1056C000581E5B18002B27D053181B1832331B7839
:1056D0008024D3185E78A023DB055F68E4033C4395
:1056E0005C60019CB606240400945F68B60EBC465C
:1056F000124F64462740009C27435F60C046243613
:1057000076008400F65A2C19B43426605E680C4C7E
:1057100034405C60031CD3E7131C313309491B7808
:10572000B4324B700423CB700F20B0230B7101F007
:10573000BFFDF7BDE40100205C090020FFFFC0FFB2
:10574000FFFFBFFFEF010020044B00225A70A0238F
:10575000DB055A7001221A707047C04620090020EC
:10576000A023DB059968064A0A40802189020A4382
:105770009A60044A0021917001229A707047C046D5
:10578000FFFFF9FF20090020024B1B68AC331868AB
:105790007047C046E4010020A023DB059868C0B232
:1057A000704730B5A023DB059B68DBB283420ED087
:1057B00001DA013300E0013BA022D2059568FF2108
:1057C0001C1C8D430C40291C21439160EEE730BD29
:1057D00038B50D4B041C1B680D1C5B183933FF33A7
:1057E0005879FFF7DEFF291C201CFFF7A7FE074BA7
:1057F00000221B681C70064B5A70A023DB055A70F0
:1058000001221A7038BDC04670010020E40100205A
:105810002009002038B50B49B3220B685200012043
:10582000B224844098541B5B0D1C141C002B01D027
:10583000FFF70CFE0020FFF72DFE2B6800221A5503
:1058400038BDC0467001002038B50B49B3220B6843
:1058500052000120B224844098541B5B0D1C141C80
:10586000002B01D0FFF7F2FD0020FFF723FE2B688D
:1058700000221A5538BDC04670010020034B1B683A
:1058800036331878400001307047C0465C0900206C
:10589000024B1B68373318787047C0465C090020FC
:1058A000054A064B12681B688D3210789B680138D8
:1058B0005843034BC0187047E4010020C003002088
:1058C00000100050064A074B12681B688D32107892
:1058D0009B6801385843044B4000C0187047C046CD
:1058E000E4010020C003002000200050064A074BBE
:1058F00012681B688D3210789B6801385843044B3E
:105900008000C0187047C046E4010020C00300209A
:1059100000400050F8B5041CFFF7E8FF0A4B196877
:105920000B685E1E0ED34A68013A09D38F68551C76
:105930005F43ED19AD0045192F68E7402F60F3E78D
:10594000331CEEE7F8BDC046C0030020064A074BF3
:1059500012681B68953210789B6801385843044BD5
:105960008000C0187047C046E4010020C00300203A
:1059700000400050F7B5FAF7ADFF344BC4301A8839
:105980000388D3180380324B1C68227853B2042B4F
:1059900024D1304B1B689A331B780093FFF7D6FF56
:1059A0002D4B02221968561E01964ED34B68013BBF
:1059B00012D38E68E518AC466A25AC44564365465A
:1059C0002D780136AC46F7186644B6003658009D6F
:1059D000BF00EE403E50EAE7019AE4E7052B24D1F0
:1059E0001C4B1B689D331B780093FFF7AFFF1A4BCE
:1059F00004221968561E019627D34B68013B12D327
:105A00008E68E518AC466A25AC44564365462D7849
:105A10000136AC46F7186644B6003658009DBF0004
:105A2000EE403E50EAE7019AE4E7002A0DD0022B4F
:105A300003D10A4B1B68373304E0032B05D1074B16
:105A40001B683D331878FFF765FFF7BD580000501D
:105A5000E401002060090020C00300205C09002050
:105A600008B5A0230120DB055870FFF713FDFFF7F1
:105A70004BFDFFF77FFF08BD08B5FFF7A9FEFFF755
:105A8000EFFF08BD08B5A0230120DB055870FFF724
:105A900011FDFFF739FDFFF76DFF08BD08B5FFF7F2
:105AA00097FEFFF7EFFF08BD054B1A68054B90689E
:105AB0001B6895331B785843034B4000C018704750
:105AC000C0030020E401002000200050054B1A68AC
:105AD000054B90681B6891331B785843034B80003B
:105AE000C0187047C0030020E401002004400050AB
:105AF00010B5A023DB051C6A0005064A000D010451
:105B000022400A431A621A6A120B120310431862E7
:105B100010BDC046FFFF00F073B5174BA0221B68F5
:105B2000D2059168D96A2C3391601C78FFF77AFA14
:105B3000124D002812D0124B124A1B7812782E6890
:105B400052B25BB20092201C1021D12201F0DBFC8A
:105B50002B68B0363060B0331B68E418002C01DAD3
:105B6000002402E0FF2C00DDFF242B68E0B2AC3300
:105B70001C60FFF716FE73BD5C090020E4010020E5
:105B8000530002005200020008B5002801D001288D
:105B900001D100F051FCFFF7BFFFFFF765FBFFF7F6
:105BA000FBFA08BD70B51F4B0D211B68A0B0DA7A57
:105BB00000230C3AD2B291425B410321C91AA023BF
:105BC000DB0558693F2210405C688022D2032243E3
:105BD0005A60421EA023D2B2DB05FF2A11D05E68B4
:105BE0003F25114C15402D0434402C435C60C046C9
:105BF0000C1C243464001C5B6D465300EC52013ACB
:105C0000E8E75968094A0A4009495A60022348707E
:105C1000CB700320B3236A460B7101F049FB20B01F
:105C200070BDC04660090020FFFFC0FFFFFFBFFF3F
:105C3000EF010020084B0948196810B5046808688E
:105C40008B6801309A00434360699B00C0180021B3
:105C500003F002FE10BDC046C0030020700100200A
:105C600038B50C4D0C4C2B68201C9A6891001A68B2
:105C700002324A43002103F0EFFDFFF745FC2B6899
:105C8000201C9A6891001A6802324A43002103F0EE
:105C9000E3FD38BDC003002000400050044B05491F
:105CA00000221A6059609A6005221A607047C04647
:105CB00010E000E0FFFFFF0010B5A023DB059C68AB
:105CC00099680C4BC9B21B68E403B0331B68E40F3E
:105CD000591AFF31E62359430134074BA040C91834
:105CE000041C0648FAF7C6FCC1B2201CFAF7C2FC35
:105CF00010BDC046E40100205C5D000040420F0082
:105D0000014B00221A60704710E000E013B50B4C05
:105D10000B48A368C01A0193FFF7CEFF094901237E
:105D20004B7004230190CB7000206F2301AA0B71EC
:105D300001F0BEFA00230198236016BD10E000E0D8
:105D4000FFFFFF00EF01002038B5051C0C1CFFF71A
:105D5000A5FF211C281CFFF73BFDA023DB0501202C
:105D60005870FFF7BDFBFFF7CFFBFFF703FEFFF710
:105D7000CDFF38BDF7B5234800F082F9FFF764FA8C
:105D8000214F0025214E224CB7421FD28036F31BF3
:105D90002026832B00DC9E100123667000203A1C15
:105DA000211CB610E370207101F082FA3B1C321CFA
:105DB000013A08D3002D04D116491868884200D052
:105DC0001D1C0433F4E7B600BF19DBE70E490422BB
:105DD0006B1A01270193E270A723211C01AA00205E
:105DE00067702371843601F063FA0423751BE37036
:105DF0000020A823211C01AA01956770237101F0DE
:105E000057FAF7BD801A06008C090020801B00207D
:105E1000EF010020CDCDCDCD10B5A023DB055C6812
:105E20008022D20322435A603F2211400A045C6858
:105E30000649214011435960C04624304000C05AF1
:105E4000034A596800B20A405A6010BDFFFFC0FF04
:105E5000FFFFBFFF08B5A023DB0559698906C90EFE
:105E6000FFF7DAFF08BD000030B58BB0051CFFF767
:105E700017FC124B6D011B6800245D19DC35201CDA
:105E8000FFF7E8FFA3000833694601345850082C97
:105E9000F5D10023181CE9580A0C02A9C958521A56
:105EA000D11752184A4001B28A4200DD90B2043341
:105EB000202BF0D100B20BB030BDC04670010020E5
:105EC00037B50024944206DA1D680134CD404543BD
:105ED0002D0C20C3F6E737BD10B5041E022C03DCE1
:105EE000FFF7F4FD640108E0FFF7F0FD044B033C0D
:105EF0001B68E4009B68E418A400001910BDC046AC
:105F0000C003002070B5041CFFF74AF80E490B6867
:105F10001B68013B11D30A685268013AF9D308683B
:105F20000A4D40682D685843ED1880182018383500
:105F30000678AD7975190570EFE7201C0021012264
:105F400000F0E8F970BDC046C00300205C090020E5
:105F5000F0B599B00492354A059312684301D318FD
:105F6000DC330393324B00241B680C8039330E1C46
:105F70001978051C4900013106A801F0B2FAFFF7B3
:105F8000C3FA211C202208A803F066FC291C01206A
:105F9000FFF772FD251C281CFFF79EFF071C0799C1
:105FA0003B1C06980822FFF78BFF059900230398F6
:105FB000FA58C0580290000C801A10AA019098500C
:105FC000088804338446019884446046088002317E
:105FD000202BECD1174908234B707C235B42CB70FC
:105FE0001920BB230B7101F063F9002310AA9A5802
:105FF000D11752184A4008A95858904200DA5A500E
:10600000944200DA141C0433202BEFD10135062D05
:10601000C1D1002334801A1CC8580433821892B2AC
:10602000202BF9D104990A8019B0F0BD700100202D
:106030005C090020EF01002038B5A023DB0599683A
:106040009D680C4B041C1B680B48B0331B68ED03A8
:10605000C91AC943E623C9B25943084BED0FC91801
:10606000FAF708FB044B01355843211C2841FAF785
:1060700001FB38BDE401002040420F005C5D0000E0
:1060800038B5A023DB0599689C680A4B051C1B6882
:106090000948B0331B68E403C91AC943E623C9B2EF
:1060A0005943064BE40FC918FAF7E4FA6843013480
:1060B000204138BDE401002040420F005C5D00003B
:1060C00008B5002807D0481006380123132900DC42
:1060D0000023C01806E00B2900DD0E39081C03213F
:1060E000FAF7C8FA08BD0000F0B5854B00261B681A
:1060F000051CDB7A0D220C3BDBB2301C9A4270414E
:1061000095B0C3B205937F4B29681B680BAC1A1C72
:106110008E3211706F689033D770311C1E7024223C
:10612000201C03F099FB784B07961A680896231CED
:1061300083CA83C383CA83C383CA83C3311C002930
:1061400000D09EE06F4B0E9E1B6803960193313387
:1061500019706B4B0E1C1B6804930BAB1F7EBF06A4
:10616000BF0E0297049F7B799E423EDA049F0598FA
:10617000BB19DF7A391CFFF7A3FF07AB1B5C9C46FA
:10618000002B15D1019B31331978013100910BA9F6
:106190000A18009911711A78111C01310092C9B2C4
:1061A00009AA11541970019B00995A18303296703F
:1061B000019A0BA993190A1812793A33013A1A7005
:1061C00001231F2F04DC039ABB401A43039206E00D
:1061D000203FBB40029F3F223B4313400293624655
:1061E000013207AB1A540136BCE70BAB039E1F7E8E
:1061F0000E963F22029E974337431F76424B1B6801
:106200001E78B606B60EFEF70DFF002809D03F4BEC
:10621000882019780236C9B2FAF72CFA4643023EB2
:1062200004D4301E3F2802DD3F2000E000206278C9
:106230001F2321789A4362703F2291431040084304
:106240002070E078696898431940031C0B43617E15
:106250002F6891436176242179432D48E370091812
:106260000023236112931393221C0B1CC1CAC1C3C8
:10627000C2CAC2C343CA43C32B68012101332B6086
:106280005DE7032902D16B6801336B60CFB2FB007D
:106290001D37DBB2FF009C46FFB200220BAB09A802
:1062A0009E18805C022901DC604400E0381801324D
:1062B0003071082AF2D1DE7868681F2296432F6871
:1062C0001040321C024324207843DA70104A013116
:1062D0001218C1CBC1C2C1CBC1C2C1CBC1C22B68D4
:1062E00001332B60062900D029E76A6801200132BA
:1062F0006A60044A12688F32137015B0F0BDC04650
:1063000060090020E40100205C0900205400020024
:1063100000800050F7B5254B00921B6800218A339E
:106320001C78234B1B689B7999423EDA0023204D51
:106330002D686E791D4DB34231DA2D68009AED1843
:106340006D78AF09E71901972427012A16D13A1C65
:10635000019F4E437A439446164AAD06AD0E171C74
:106360006744AC46C518AD5D01973F2D00DD3F2564
:10637000019AEDB2161C664435770EE03A1C019F77
:1063800076007A4394460B4AAD064E439444AD0ED4
:1063900065442D7F5F00BE1985550133C7E72B6823
:1063A00001318C331B78E418BBE7F7BDE401002012
:1063B0006009002000800050F0B585B003F022F99C
:1063C0001A4B022419680B1C92331A78184B1F6859
:1063D00024235343174E9E190396031CBD691E1AAE
:1063E000AE421ADA1D788E190295767EB50912D161
:1063F000B606B60E0196029E75B23F2D01DD3F2511
:1064000002E0EE43F6173540EDB2019EAC46039D27
:10641000AD1966462E770133E0E70B1C94331B78E9
:10642000013CD218002CD3D105B0F0BDE40100200E
:10643000C003002000800050F0B5BB4BABB01B6820
:1064400000240193DB7A0D220C3BDBB2271C9A421D
:1064500067410CA8211C0C2203F0FEF9019D089451
:1064600009946D7903260295019DF61BFFB2019AEE
:106470000298AB1A834213DAE97A381CFFF720FE40
:10648000072801D90020FFE208A90B5C0135B342BF
:10649000F8DC0133DBB20B549C42E8DA1C1CE6E763
:1064A0000122019D0C92A879002181420ADA131C75
:1064B0009D1AA54203DA372BE4DC0133F8E70131FA
:1064C0001A1CF2E7352ADDDC00250223019E0C951B
:1064D0000D93F27A2F1C0C3AD2B20D2191426F41EA
:1064E000924A0326F61BFCB2176803943A1C8A32C0
:1064F0000FAC1570291CD370201C6C22029603F07F
:10650000ABF98B4B0A951A680B95231C61CA61C3C2
:1065100062CA62C323CA23C3012124234B43221C22
:10652000E31861CA61C361CA61C361CA61C3029EE3
:106530000131B142F1DB00240294019D6B799C4250
:106540004ADA019D03982B19DD7A291CFFF7B8FD63
:106550000AAB1E5C24217143B446661C05960A18DA
:106560000FAEB6180496049A059E16711F2D08DC0E
:106570000FAB59180123CE68AB401D1C3543CD60CD
:1065800011E01B5C24225A430FA9203D01238A18E5
:10659000AB401D1C137E9906890E0D433F210D4013
:1065A0008B431D4315763F23051C3A191D40567831
:1065B00004956546A901049D9E4335431D406346ED
:1065C00029430133029E5170DBB20AAA13549E4242
:1065D00000DA02930134B0E73B1C029E8C330027A3
:1065E0001E700197504B019E1B689A79964200DB02
:1065F000A4E0019C0D9D1B190433D87F1F231D406F
:10660000AC46051C0123203D1F1CAB401D1C029BFA
:106610003F221540013B242253432AAEF318029A2D
:1066200087405C3B013A1CD3242151430FAC6118D5
:10663000CC781F26B44366463443CC7000241C60DB
:1066400018314E783F24A6434E701F2803DC19688A
:106650003943196003E04E78A6432E434E70243B25
:10666000E0E7334B019F1B681C78DA195032A4060F
:106670009579A40EFEF7D6FC002813D02D4E882065
:1066800031780135C9B2F9F7F5FF31784543C9B220
:106690008820F9F7EFFF02344443013D023C00211A
:1066A000681C03D0291E1F2900DD1F213F2C02DD9D
:1066B0003F22039203E0E343DB171C4003940022D4
:1066C000029CA24228DA24252C1C54430FA81F2622
:1066D0000F1C0319374004975F78B7433E1C049F93
:1066E00037435F70039F3F2637400497275CB743CB
:1066F0003E1C049F374327540C9C372C23DC6543F6
:106700000D4801344019E0CBE0C0E0CBE0C00132DD
:10671000E0CBE0C00C94D3E7019D0D9B0135013324
:1067200001950D935EE7C04660090020E40100205A
:106730005C0900205400020000800050D34B0C9FE5
:106740001B688B331F700D9C00260CA80D96FFF75D
:10675000CBFC0D94CD4C311C20680422823003F018
:106760007BF82068311C0422863003F075F8256818
:106770000C982A1CC3B28232137053701371537178
:10678000C34A341C12680D210192D27A0D980C3A3A
:10679000D2B2914274412A1CE7B29232137005972B
:1067A0002B1C03273F1B95330FAC311C18706C2238
:1067B000201C029703F050F8019B0A960B96643355
:1067C000221CC2CBC2C243CB43C283CB83C20121B2
:1067D00024234B43221CE318C1CAC1C3C1CAC1C38D
:1067E000C1CAC1C3029E0131B142F1DB237EE76819
:1067F0009B069B0E039704930024019E73799C4291
:106800003DDA019E05983319DB7A191C0293FFF7D4
:1068100057FC0AAB1B5C9C46002B03D10FAF631CDB
:106820003A1813710FAE3218127929190B1C6A33FA
:10683000013A1A704E7E3F239E430AAA0696165CC2
:10684000071CB6010796069E1F403743079E1F4050
:106850003E43029F4E7601211F2F04DC039EB94068
:106860000E43039606E0029E049F203EB14039434A
:10687000194004916346013313540134BDE70FAB53
:106880001A7E3F21049C039F8A432243129794352A
:106890001A7601232B70B279032313407D4ADB0063
:1068A000D31800250593019500220FAB1392597E52
:1068B0003F20814359767649059D0968019E1492CF
:1068C000AC5902910D9D88795E7E1F210D40D978CB
:1068D000B606C3071B1A071FC906B60E0395069313
:1068E0000797C90EB4460492151C131C83423ADA6A
:1068F000029E5F00F11823310978032B06DD079F04
:106900009F4208DC069F1037FF187F00261C3E417F
:10691000371C032604E01F1D261C3E41371C0126A0
:106920003E40012E0CD11F2902DC8E40324317E07D
:10693000203967468E403E433F273E40B4460FE035
:10694000002E0DD101261F2905DC8E40311C049E2E
:106950000E43049604E020398E4035433F273D40E6
:1069600001330399C2E70FACE6781F239E43194019
:106970003143667E3F239E4367463E436676E17021
:10698000049922616161A17E99430D43424BA57632
:106990001B681818029B503064331E788579B60640
:1069A000B60EFEF73FFB002813D03C4F8820397805
:1069B0000135C9B2F9F75EFE39784543C9B288207E
:1069C000F9F758FE02364643013D023E00236A1C99
:1069D00003D02B1E1F2B00DD1F233F2E00DD3F2683
:1069E00061781F22914313400B436370F343227875
:1069F000DB171E403F230C999A431E401643242266
:106A00004A43274B2670D218131CE0CCE0C325CC98
:106A100025C3C1CCC1C30D9A019C4B1C0132043467
:106A20000C930D920194082C00D03DE7174C22687E
:106A300093321370FFF7C0FC23681A1C8A32117856
:106A40000532D17210781C1C10739C34013A1278F4
:106A50006070181CA83022700270013242701A1C3B
:106A60009E3211701D380078191C9F3108701288F1
:106A700001310A800E391A1C0978A23211700F3ABE
:106A80001278A3331A7001202BB0F0BDE40100206E
:106A900060090020C09800005C090020540002003A
:106AA0000080005030B50E4B1B689979884203DA9C
:106AB0001B180433D87F12E05A798D18411AA84266
:106AC00002DA5B18D87A0AE09C7A8A1A2D19A84251
:106AD00001DA9B1801E0141B1B193833D87830BD3C
:106AE00060090020F0B5A024E405A368AF4BA5B071
:106AF0001B6800AF59799A7968468A18597A9B7A47
:106B00005218D3181A1C5A43BB62D31DDB08DB0092
:106B1000C01A85466D46FF21BD6102F09DFEFF2033
:106B2000FFF7AEFABD6AA24BED001B1ABB602B1C2F
:106B30000E33DB08DB006846C01A85467D616D4672
:106B40007D62BD6AAD002B1C0A33DB08DB00C01A76
:106B500000220023BA63FB633D613862E268954B13
:106B600085461340E360BD6A013DFD602C1C601C3E
:106B700017D0201CFFF796FF011C381C7030202214
:106B800002F00AFE386F9021C9198300CB187A6F82
:106B9000583B01211D6891400A1C2A431A60013CA0
:106BA000E5E7BD69FD610025FD62FD6AB86A8542C1
:106BB00000DBDAE000217A69786A02F04DFEA02459
:106BC00000213A69386A02F047FEE4050023236396
:106BD000636B3F26B3436363BD6BA563F86BC0B2C1
:106BE000786330403863E36BB3430343E36364206B
:106BF000FFF746FAFEF728FBF86AFFF753FFC1B22A
:106C0000381C5430202202F0C7FDB96BFA6BBB6D03
:106C100039647A647A6D0121994090200B1CC01967
:106C200091004118081C503802689A430260786D40
:106C3000131C002808D058390A685340626B33404F
:106C4000B2431343636301E06B402363A024E40574
:106C5000A563E36B396B3F26B3430B43E3630A2021
:106C6000FFF70EFAFEF7F0FAE26B80235B001343A6
:106C7000E3633A6C5540A5637B6C7A6B5A40E36BD7
:106C80003240B3431343E363FFF708F87D6C3E6C77
:106C90007B6AAC460124484ABD689168A94214DB6E
:106CA000464A65461068526830402A405D68954201
:106CB00003D3F0D11D688542EDD23D6ADA60A200AF
:106CC0009860A95001340833E5E7FFF719F8A023CD
:106CD000DB05D96B3A4A0A40DA63012C3DD0651EC8
:106CE000786AED004519013C002C36D02B1C083B7E
:106CF0001A6829685B6891436A68FE689A43A30032
:106D0000B964FA647B63FA6A964224D0301CFFF7B8
:106D1000C9FE011C381C7030202202F03DFD7B6F43
:106D20000122386F9A409021131CC91982008A18D9
:106D3000483A12681A420CD07B6B3A6A1720D25834
:106D4000404250431F4BC018FEF7B6FFF9690011CF
:106D50008855013ED7E7083DC5E7FD6AB86A0135A9
:106D6000FD62FD692D18FD611FE7381C00211A2204
:106D7000543002F071FDBD6A3C1C7034EBB22370DC
:106D80006370A370381C0023391CE37023711A222E
:106D9000012354317630637102F01CFD201CB96967
:106DA00000F0F8F9BD4625B0F0BDC04660090020EE
:106DB000FFFFFF00FFFF0FFF10E000E0400000506A
:106DC000FFFEFFFFE9FFFF16014B18607047C0464A
:106DD00068090020014B18607047C0466409002014
:106DE000F8B5F9F765FD041C01F088F8051CFEF7FD
:106DF000BFF8394E211C071C1022306802F0EAFC53
:106E00002B88346823741B0A6374AB88A3741B0A31
:106E1000E374324B1B680533DB7F002B03D0BB7957
:106E200023757B7902E07B792375BB796375FB79E8
:106E30002F1CA3752B1C683319886A370B0AE17560
:106E400023763B78286863767B78A3760A235843B9
:106E5000F9F710FCE07668680A2339885843F9F797
:106E600009FC20771E4C7569231C0833B3601D4B49
:106E700074601B782B70FEF7B1F8627E217E1202DF
:106E80000A43A17EE87109040A43E17EF36809061A
:106E90000A43110A1A705970110C120EDA70627FCF
:106EA0009970217F12020A43A17F09040A43E17FFE
:106EB00009060A43110A1A715971110C120EDA717E
:106EC000221C2C322D3499711178227812020A4337
:106ED0001A72120A5A72F8BD18030020C00300206B
:106EE000D0BF000047000050F0B58BB0F9F7E0FCD0
:106EF0001B4BC26C5B68002459685A60194B9D6833
:106F000002F060FB6860FFF76BFF174B174A1868C9
:106F1000174B1B681D882B0A057143716B46C2CA4B
:106F2000C2C3C2CAC2C3C2CAC2C3126869461A6017
:106F3000AD006B58012283710E4B5A709C7002F0A9
:106F40003BFB0D4B58600D4B1B78A34205D00C4BFF
:106F50005B681C705C709C70DC700BB0F0BDC04650
:106F6000B4030020340200200C030020E09800004D
:106F7000680900203002002098050020A0050020AC
:106F8000F402002008B5084A51684B780749DBB283
:106F90000B70012B05D0022B05D1136801225A700A
:106FA00001E0FEF723FA08BDB40300206B050020C2
:106FB00008B50A4B1B78012B06D0022B06D1084BD3
:106FC00000221B685A7001E0FEF722FA054B7F2170
:106FD0005B681A788A431A7008BDC0466B050020AA
:106FE000B40300200C030020F8B5194D0024194EFD
:106FF0003378012B08D0002B19D0022B18D1164B57
:107000001B685C78E4B213E0FEF712FA041C002D52
:107010000BD1FEF7FDF92E23FF33013B002B01D0EE
:10702000C046FAE7FEF7E2F9094D013D00E01C1CFD
:10703000094F7A68537832789A4206D0FFF7B8FF42
:107040007B68044A5B78137001E0002CCFD1F8BD57
:10705000FF2C01006B050020B403002037B50E4B58
:1070600000931D1CFEF7E4F9009B041C002B0CD1BF
:10707000FEF7CEF9094B0193019B002B02D0019B37
:10708000013BF8E7FEF7B2F90095009B013B009346
:10709000002CE7D137BDC046563F0000560603001E
:1070A000024B5B681878C0B27047C046B40300203A
:1070B000024B5B689878C0B27047C046B4030020AA
:1070C000014B5B6898707047B4030020024B5B680B
:1070D000D878C0B27047C046B4030020024B5B684A
:1070E000587AC0B27047C046B4030020024B5B68B8
:1070F000987AC0B27047C046B4030020024B5B6868
:10710000587BC0B27047C046B403002008B5044B9A
:10711000002158680A22163002F09EFB08BDC046C6
:10712000B40300200023042806D8044B08305B6811
:1071300040001818C3889BB218B27047B4030020EF
:10714000074B021C08325B685200042803D89A18C7
:10715000D388D18003E09B18DA880022DA80704758
:10716000B4030020014B5B6858757047B4030020DE
:10717000034BA0221B681A701A78A02AFCD0704713
:10718000B4030020024B5B681878C0B27047C04659
:10719000940300200F4A30B55368FF241C709060A0
:1071A0000D4A04781160817805794C43417964195E
:1071B0004906490E6143094A92681160084AA021B4
:1071C0001068017051681A78FF2A02D10A78022AE1
:1071D000F9D030BD9403002098050020340200202F
:1071E000B4030020014B1B68188870476809002011
:1071F00008B5FFF7F9FE024B00221A6008BDC04631
:107200006C05002070B5074B074C1A682668011CF6
:10721000957998682A1C8019751902F0DBFA2560A7
:1072200070BDC0460C0300206C05002008B5074B5C
:107230001B68002B09D0064ADBB252687F21194037
:107240001170044A9370FFF79DFE08BD6C05002085
:107250000C0300203002002070B5114B1A68B023D7
:107260005B00D35C022B06D1FFF7BEFEFFF78AFE60
:10727000FFF7BAFE13E00B4A8026536876421D786A
:107280007F242E43C9B2F6B20D1CA6432540341C00
:107290002C431C70044B90609970FFF773FE70BD17
:1072A000700100200C030020300200207047000015
:1072B00070B5154C63681D79EDB2012D22D1854062
:1072C00058781E78000230439E7836043043DE78CA
:1072D00036063043284215D0FF2018710B48A160B4
:1072E000026088780C78C97860434906490E4143AA
:1072F000074A92681160074A7721126811701A795B
:10730000FF2AFCD070BDC046F40200209805002082
:1073100034020020B4030020014B1B6858797047E9
:107320002C020020024B00221B685A717047C04695
:107330002C020020014B1B68187870472C0200209B
:10734000014B1B68187070472C020020014B1B6812
:10735000987970472C020020014B1B689878704781
:107360002C020020014B1B68987070472C020020F3
:10737000014B1B68187970472C020020024B5B6997
:107380001872000A587270471803002070470000F6
:10739000002303600B60284BF7B59A424ADC1312B6
:1073A000122B34D8254C9B001C59254B9A420CD1EA
:1073B000244D6B685E781F7836023E439F78DB78F9
:1073C0003F043E431B063343AB60002C32D0E368DE
:1073D000013B5D1C2ED0D5B2019565681E1CEF5C8B
:1073E000019D013BED1BF4D42768B300DB59002B52
:1073F00020D0A268925D521B0A60002A02DD5D194E
:10740000056017E0104B03605B780B6012E00F4CD7
:10741000E3686668251C013B0CD35C00345B141BDD
:10742000F9D42E689B00F25812190260AA68D3584A
:107430001C1B0C60F7BDC046FFEF0000A802002037
:1074400014130000000300209602002034020020E4
:1074500008B5C023DB00984207D10C4B1B681A7893
:10746000052A12D005221A700FE0094B84225B68AE
:1074700092001B785B065B0E9B18984202D1FFF7C7
:1074800097FD02E0034B9842F9D008BDB4030020F9
:107490000C030020030E0000031E1F2B09DC102824
:1074A0001DDA072819DC042815DA0120022B17DA67
:1074B0000FE07F2805DCC0170022402B504105302B
:1074C0000EE00720FF2B0BDD802292000820934264
:1074D00006DD002004E0022002E0032000E004209A
:1074E000704770B5041C081C0E1CFFF7D5FF031C69
:1074F000051C10330120311C9840F9F7BBF82060BF
:107500006560201C70BD38B5051C1C1C181C8D4204
:1075100009DB0498954206DAC01A6D1A6843511ABD
:10752000F9F7A8F8201838BDF8B501254E1E6C00F3
:10753000B54202DA165FB0420CDAA61E1D5F115F7B
:107540009B5F401AEB1A5843935FC91AF9F792F8F8
:107550004019F8BD0135E9E770B501244D1EAC4274
:1075600002DA155DA8420CDA661E1D5D115D9B5D99
:10757000401AEB1A5843935DC91AF9F77BF8401982
:1075800070BD0134EAE70000014B18607047C04647
:1075900074090020014B18687047C0467409002028
:1075A000014B18607047C0466C090020014B1868F9
:1075B0007047C0466C090020014B18607047C046F8
:1075C00070090020014B18687047C046C4030020B2
:1075D000F7B55301161C224A009014680191E41873
:1075E000DC3400212022201C02F036F90120311C5D
:1075F000FEF742FA0025281CFEF76EFC0023E15836
:10760000C758CA19E2500433202BF8D10135062D92
:10761000F1D1002560590621F8F7DEFF60510435ED
:10762000202DF7D1231C009801990822FEF748FC71
:107630000023E1580A04E2500433202BF9D1094D0C
:107640001023AB7108236B70243E0423291C0020F7
:10765000221CEB702E71FFF72BFE0023AB71F7BDE0
:1076600070010020EF010020F0B587B00E1C051C52
:10767000FDF79CFC2B49041C00204F23021C0B71BE
:10768000FFF716FE284B29491A68096853680191CB
:107690000020013B18D3E1183A310F780199BF005F
:1076A00037310978BF59CF401168BC464F1E00974B
:1076B000EFD39768794359180131890049596746D2
:1076C000C91B40180099F1E7D168F8F7D3FF184EAD
:1076D000051C3368DF89174B1B685988781AC0036B
:1076E000691AF8F7C7FFFA23041C1B02984200DD51
:1076F0001C1C114903234B707C235B42CB70002080
:10770000502303AA0B71039704950594FFF7D0FD4E
:107710003368DB89002B01D180242402A0B207B09A
:10772000F0BDC046CB040020C00300205C0900204F
:10773000740900206C090020EF01002038B50C1CF2
:10774000051C02F01BF80B4B64211B6808341B79E5
:107750005943094B69431B6821411B7B002B07D010
:10776000064B04301B6840001818C3885943C913DE
:10777000081C38BD6C09002074090020C4030020D7
:10778000F8B5151C041C01F0F9FF1C4B64271B689D
:10779000061C1B795F43FEF771F84743FEF778F844
:1077A000174A07411268381C127B002A08D0154A74
:1077B0000436126876009619F288131C7B43D8139E
:1077C000211CF8F757FF104B041E9C4200DD1C1CC7
:1077D000FDF7ECFB0D4B03211A68DC32101C002373
:1077E000EE5E076866430233BE1B40C0102BF7D124
:1077F000013920320029F1D1F8BDC0466C090020C2
:1078000074090020C403002033B30000700100207D
:10781000F7B58027264D0E1C00233F06F25E254952
:107820004A431214F252954200DD151C974200DAC9
:10783000171C0233102BF1D11F497E2308225B4213
:107840004A70CB701920BC23321C0B71FFF730FD3E
:107850001A4CEF23211C13206A46237100950197CF
:10786000FFF726FD164C0F3501DB0F2F02DD00233D
:10787000236009E023680A2B06DD124B08211B68F0
:10788000321C1868FFF77CFF0C4A21680023019323
:10789000F023137100911320111C6A46FFF708FDB5
:1078A000236803498B4201D001332360F7BDC046F2
:1078B000FFFFFF7FAA2A0000EF010020E80100205F
:1078C000F805002070010020F0B51C4E85B0366828
:1078D00001ACFC36F76E366F002501956760A66037
:1078E000AA420BD19B001B59824225DA54001D5B32
:1078F0000C8801322C190C800231F5E79200002B24
:107900000AD1A258834217DA5C000D88145B013358
:107910002C1B0C800231F5E79B00A6581C592A1C31
:107920002B1C824208DAE75ACD5A01327D19F75AE8
:10793000ED1BCD520233F4E705B0F0BD700100201D
:10794000F0B585B00392304A02901268DC69527932
:107950000D1C9440002C00DC0124FDF78FFF061C59
:10796000FDF796FF011C301CFFF7E8FE0A99604303
:10797000F8F780FE002807D124490020ED23021CDF
:107980000B71FFF795FCF7E7E62800DDE620029E85
:10799000002101961E4B1B681A68914223DA019B55
:1079A0002A1C00241A4F01933E68151CB4467668C1
:1079B0004F1CB44215DA157801956546AE687E43D2
:1079C000A619039F01367600F65F019F4643BD1B53
:1079D00015701E882D12AD191D800134013202333D
:1079E000E0E7391CD6E70B491B790A704B708B70A6
:1079F0007E235B42CB7004206023029A0B71FFF759
:107A000057FC012005B0F0BD6C090020CB0400201C
:107A1000C0030020C4040020F0B5354E89B033689F
:107A200004AF7960FA6059681A68023102324A4339
:107A30005200131C0833DB08DB00B8606846C01A2C
:107A4000854604AC0021201C01F006FF294D0021D1
:107A500028682C22303001F0FFFE33686846196830
:107A60005B684A001032D2085B00D2001033801AE3
:107A7000DB088546DB00C01A04AA2B688546043261
:107A8000B868191CDB69019205AA00900292303196
:107A9000FA68201CFCF712FC336817491A68F86072
:107AA0000A709A6858688A707E2301325B425200DD
:107AB0004870CB7001205323A2180B71FFF7F8FB1D
:107AC000F9680020814210D10C4BFA201B6880001D
:107AD000D98EF8F7CFFD2D6800903035B8687968F9
:107AE000221C2B1CFFF72CFF0120BD4605B0F0BD6A
:107AF000C003002070010020C404002038090020C9
:107B0000F7B5104B00901D6801912A68561E17D3D7
:107B10006B6800981C1C7443E41864000419023C50
:107B2000013B0BD3AF6801995743DF190137BF0001
:107B300078582788844667442780F0E7321CE5E7B9
:107B4000F7BDC046C0030020F8B5141C0E1C071C6E
:107B50001D1CFDF72BFA221C363210782A1C3732F6
:107B60001278363540003B88297801309040373410
:107B700058434900237801319940F8F77BFD308064
:107B8000F8BD0000F0B589B00792254A0590166847
:107B9000244A3468126806910392234A12680492B8
:107BA0006A22FF325343214A1268D2180292221CE1
:107BB000013A32D373681E4F181C50435D1E654353
:107BC000D91909180090029F0598490055194118C4
:107BD0007D19013BECD30027C85F069F3841039F06
:107BE0003F7B002F15D0079F7843C0130190B02032
:107BF00047000498C05D022801D12F7805E0029863
:107C00008446009884446746FF5C381C019F784393
:107C1000801108802D1B0239DBE709B0F0BDC0469A
:107C2000C0030020740900207001002070090020AA
:107C3000FFFFFF7FF0B57C4F91B03B6809917B4916
:107C40000D92596080210022090699600F921A60F6
:107C5000774B784E1A68B0235B00D35C764C0A935E
:107C60003368051C996958699A680423E370A02356
:107C7000A27023710132099B92009A1820706170E2
:107C80000220211CFFF714FB36686C4B70690F99BA
:107C90001B683A680691059008930490211C049C87
:107CA000B369013C07944DD3079C059F5C435F4338
:107CB0005E48A4461C18E019400064460197281845
:107CC0000D9F0290A00038180C90019864004700A6
:107CD0007F420B97A446013B31D30C9F9C003C593B
:107CE000B768200C049C6743DF19099C0137BF006B
:107CF0003F59C41B5768BC4200DA54609068844204
:107D000000DD94600B98029F3F1860463C52089833
:107D1000E7170078E4197C4084420CDB029807885E
:107D20003F190780176808983F1917600078069F69
:107D3000241A3F190697029802380290CBE7079B56
:107D40000493ACE7069EDBB2059A4B708B70CB7840
:107D50000F9601327F260A70B34302228024134318
:107D600064422343CB701A20A1232A1C0B71FFF716
:107D70009FFA33490422CB780127B34313431C43B2
:107D80001A20CC230FAACC700B714F70FFF790FA1A
:107D90000A9C2A4B022C39D1264A1B68146804938A
:107DA000A0690021031CFF22049F7F880597013BE7
:107DB00011D366694643B4469C4467467F007E5FA4
:107DC000B446059EB445EFDB994200DAD9B29A4237
:107DD000EADDDAB2E8E70F9BBB421FDD636954B20C
:107DE000434348B2001BC40F241864101419E4B2B2
:107DF000E418D21852006400505F2A5F90420FDDF1
:107E0000CB185B005B5F93420ADD0AE01B680F99A9
:107E10005B88994200DC0027F8B202E0002000E015
:107E2000012011B0F0BDC046C4030020FFFFFF7F5A
:107E300070010020C0030020C40400207409002049
:107E4000EF010020F7B5264B264D161C1A682B684B
:107E50000090019110689969F8F7BEFB224B041C51
:107E60001B685B799C40002C00DC0124FDF706FDBB
:107E7000071CFDF70DFD011C381CFFF75FFC311CD2
:107E80006043F8F7F7FB2D686C69221CAB69013A77
:107E900014D31F1C5743009EF91889007118019EC6
:107EA0007F00F619B4460439013BEFD367465E0004
:107EB000BE5F0F684643BE1B0E60F4E70B4DDBB29E
:107EC0001022AA716B70AB7004206023291C009AE9
:107ED0002B712C70E870FFF7EBF90023AB71F7BD45
:107EE000C4030020C00300206C090020C40400204B
:107EF000014B18607047C0467C090020014B186890
:107F00007047C0467C09002008B5054B1860808A80
:107F1000FFF734FA0020FFF739FA01F067FA08BDDD
:107F200078090020014B18687047C0467809002086
:107F3000014B18687047C046C8030020F7B5324CA3
:107F4000C6252068C722AD0000219200465901F0E5
:107F500083FC2E4B24681F686651BA68F96850008C
:107F6000401A00024900F8F785FB3B697969061C55
:107F7000A0605800401A00024900F8F77BFB244B30
:107F8000E0601B6876005A681D68013A013D1202E4
:107F900040002D02B6184519053326616561D97F69
:107FA0003A1C3B1C6A336832002903D012881F88B0
:107FB000019202E01B8817880193311C3804F8F7FE
:107FC00059FB019A291CA0631004F8F753FB0A23FC
:107FD0005F43311CE0633804F8F74CFB019B0A2235
:107FE0005A43291C206510040192F8F743FB391C01
:107FF00060653004F8F73EFB0199A0652804F8F7A6
:1080000039FBE065F7BDC046C80300207C090020AD
:10801000C003002010B502248B7804575AB2944252
:1080200000DD8370CB78032404575AB2944200DAFF
:10803000C3700B78002404575AB2944200DD0370D9
:108040004B78012141565AB2914200DA437010BD7B
:10805000F0B58DB00792079C089301322301C41834
:108060000B920A912589089E2FB204953501451976
:108070002E892368069636B2B819099028687B4382
:1080800070430999C018F8F7F5FA696863684E43B8
:108090007B4300B209992060F018F8F7EBFA00B2C0
:1080A0006060201C129904220A3001F093FB069EA6
:1080B000049FF319238100232B81089F079D0A9EAB
:1080C000AD00BA00AC46331CB118634408880027E1
:1080D000DE5F05B2AE4204DA1880C878D8708978BD
:1080E00099708649089B09680133C86A0125834253
:1080F0000ADA149E9D40311CB75861440E683D4019
:1081000035430D600133F1E7149F0023BB50089EF7
:10811000079F291CB140BD40149A0495CE43089F87
:10812000BB421ADA1068014214D0079DAB4203DA51
:10813000049F384310600AE0079DAB4207DD149F9F
:10814000381C6044056801279F402F430760106872
:108150003040106001330432E1E7129D2D786DB29A
:108160000495129D0123EB56049E9E4200DD9FE084
:10817000129EB67876B20596129E0322049BB256E2
:10818000059F0133974200DD90E05C4A059D12682F
:10819000139E9768D06A7B4301335B190697F718E3
:1081A0003B780990013B9C461B1A012B7ADD01218B
:1081B000052349420020013B002B2BD0504D0126C6
:1081C000ED187642AE57049DAE19069D01367543F3
:1081D00002954C4D139EED18013D2D786DB2019521
:1081E000059D7619029D7619019D76197578013DD8
:1081F000E1D3099EB542DEDA079EB54202D0089E61
:10820000B542D8D14E1C03D0A942D4D00120D2E728
:10821000291CD0E7002845D0136B9C4540D10B9D0D
:108220003D700527013F002F3CD0364B0121DB1963
:1082300049425956324B0122DB1952429A56049D4B
:108240002E4B059EAA181D687118AE68531C734307
:10825000139E01335B18F0180678002EE2D1159EAC
:108260005B009B5B002BDDD02D6B5943057025898E
:1082700020682EB270430902401861685A435D19A4
:108280004E43ADB225812DB21202291CB618F8F763
:10829000F1F9291C2060301CF8F7ECF96060C1E7A7
:1082A00062463A70059D0135059565E7049358E7E8
:1082B0000022AA56129C0123E3569A421BDC129F0D
:1082C0000223FB56129F03203856511C834210DCB8
:1082D0000A48139C0068089D806841430131C91811
:1082E000611808780138A84201D10B9E0E70013345
:1082F000E8E70A1CDEE70DB0F0BDC046C003002071
:10830000C6990000BE990000F0B5A7B02C9C0C9255
:10831000009412930A901791FBF744FFFFF702FEB7
:10832000CA4B1A68B0235B00D35C012B04D1418D8A
:10833000828DC48D038E0BE0C54B1B681A1CEC327A
:10834000181C1188F0300232F233128804881B881E
:10835000C0480068456C012D05D1006C012802DD84
:108360001494159301E014911592BB4B1B68DB6AC2
:108370005F1E7B1E002F00D176E1129E9A0092595B
:108380000697FA400E921F1C0E9E002EF1D0B24BA3
:10839000069C1B68DB6A9C42EBDA0E9C01221442AD
:1083A00000D14CE10A9E3D017519069E28683401F2
:1083B0000A9E341923686E68C11A6068331AC81798
:1083C0000E184640D8170F961E1846400F980B9669
:1083D000B04202DD1092180203E000260802109657
:1083E000191CF8F747F91CAE211C042211900A3120
:1083F000301C01F0EFF9291C301C0A31FFF70AFE8E
:108400002868236820900822A15E0D930791082216
:10841000A95E079B0891CB180D9A09930799089BB1
:10842000484353430999C018F8F724F90D9B646831
:10843000219022936868089B079D634323906843BB
:108440000999C018F8F716F92594249000211DA861
:108450000C22002401F000FA3457012508947557C6
:108460000224189534577C4B1994F6781B6876B221
:108470001A960D93089C189DAC4200DDA2E0089D61
:10848000199E2D0216950796089B079D1A9E01338B
:10849000B54200DD94E00D98079C80680C9D434335
:1084A00001331B190D9E0593EB5CF16A013B0990AA
:1084B0008B4246DB0024012005224042A446013ABB
:1084C000002A2CD0654E0125B6186D427557089EBE
:1084D0007519099E01356E431396614E0C9DB618B1
:1084E000013E367876B20496079EAD19139EAD19FB
:1084F000049EAD196E78013EE1D38E42DFDABE42B2
:1085000002D0069DAE4206D1451C06D0B042D6D060
:108510000126B446D3E70124D1E7301CCFE7013070
:108520004AD0059865464200002D01D1002C02D1A9
:108530002C9EB05A10E02C9C591AA05AF8F79AF8C1
:108540000AE0002B38DBBB4202D0069DAB4233D1A0
:10855000059E2C9C7300185B00282DD0079D0323DB
:108560002902013B28D3109D20AC23AA9E00002D98
:1085700009D09559169A551B119A5543A2592D1297
:10858000551B6D1A08E0A559119C4D1B6543925966
:108590002D12169E551BAD1BEA17AD185540FF2D29
:1085A000DFDC80267600751B45439C001DAAA6587B
:1085B0002D127519A550D4E7079C0134079463E781
:1085C000089357E71F9B1D9C9C4200DD1C1C109EBE
:1085D000002E06D10B9D331C002D0CD00F9E0F9545
:1085E0000B960B9D0F99A801F8F744F83F2800DD82
:1085F0003F201C4B1B5C2D21149E159DC81A7043F7
:108600006B43C018F8F736F844431E9BA412A342EC
:1086100015DD069EBE4201DB0697371C0C9C129DA1
:108620002C9E1CAB009301943B1C029503960A9868
:108630001799069AFFF70CFD3B1C069F0693069CB4
:108640000E9D01346D0806940E959DE67001002084
:108650007C090020C8030020C0030020C699000048
:10866000BE990000CE990000244E01213068494295
:1086700007641022183001F0EFF83D1C3C1C371C39
:108680001F4B1B68DA6A944224DA0A98260186197D
:108690000821735E002B1ADD3B681A6C01321A64E4
:1086A0001B191D76A54210D00A9A336871682801FB
:1086B0001018416003603389311C03810A310A308C
:1086C000042201F087F8002333810135EDB2013433
:1086D000E4B2D5E70B499A680C9E1C685D688A7005
:1086E00001230132CB70B218302306200C704D707C
:1086F0000B71FEF7DDFD27B0F0BDC046C8030020BA
:10870000C0030020C404002038B5144BC2171B68F6
:10871000841854409A6BDD6B5443CA178918514032
:108720004D4324142D14AC4202DB231C2C1C1D1CB5
:10873000A001291CF7F79EFF094B1B5C281C002B8E
:108740000BD05A21074AC91A49008D5A5B00684369
:108750009D5A00146C432414001938BDC80300202E
:10876000CE99000008990000F0B58FB000AFFB6013
:10877000794B7A611B68B961DA6AFB62D31DDB0849
:108780005400DB006946C91A231C0833DB08DB00F0
:108790008D466E46C91A3E638D46B9620121386224
:1087A0004942386B01F058F8B86AFF21221C01F0E9
:1087B00053F86A4B00261B687B62F96A096A8E428D
:1087C0004FDA7969F300CB1804229B5E002B45D069
:1087D000331C796A8C339B005A58C6239B00CB58B4
:1087E0005200D3180A6CF9687B63B300CB180124DC
:1087F0003A61FB61644200253B699D421ADA3A6A9C
:108800002B01D31808215A5E002A10D0FA69196882
:108810000020105E081AF96902228A5E5968891AD6
:10882000FFF772FF7A6B904201DA2C1C78630135F6
:10883000EDB2E1E7611C11D03B6B1A5763000132C6
:1088400007D0B96ACB181A88796B8A4206D9198081
:1088500002E07A6BB96ACA523B6B1E550136F6B21A
:10886000ABE700243D4B1D682A6C944220DA3A6B3A
:10887000165D73B2013318D0F6B20E2070433A6A17
:10888000BB692101511818184A680B68428003809F
:108890000B89042283800A31083000F09BFFB96AFB
:1088A00063008C365B5AB60073510134E4B2D9E7E9
:1088B0000024286C844233DA3E6B335701332CD1C9
:1088C0003E6A2101711808228B5E002B25D0FE6ABA
:1088D000336A9C46002363451FDA7E69D80030184E
:1088E0000422805E002815D10E205843BE6930183E
:1088F0000422865E002E0DD13E6B33550A684B680C
:10890000028043800B89042283800A31083000F002
:1089100061FF02E00133DBB2DDE70134E4B2C8E716
:108920000023F96AFE6AC96A326A8B420BDAE918D7
:108930000C7E944202DA3E6B325D00E0FF2201338E
:108940000A76DBB2EDE7031E934200DD131CBD4641
:108950002B640FB0F0BDC046C0030020C803002048
:10896000F0B595B0041C08910992FFF7E1FA734B3A
:108970000A901B681B6A5F1E0E237B43E418261DAA
:10898000791C00D1D7E00021735E002B00DCCFE022
:108990000723F3560622B2560B93684B002418683F
:1089A000674B94461B6804940D9305940B998C4572
:1089B00069DC05257557614604220902B2560C95FB
:1089C0000E910C9D63460133AA425ADC8468551C03
:1089D000291C61430394089CC9180695635CC56A09
:1089E000AB4226DD0523013B002B30D0554D039CC7
:1089F000ED18013D2D786DB20795534DED18013DF1
:108A00002D786DB2551901356C43089D02942C1CCC
:108A1000079D644465190F94029C2C196578002DFC
:108A2000E1D00D9C6DB26519ED7D6DB2BD42DAD11C
:108A300008E0002B0ADD0A9CE31817241C570023CA
:108A4000BC4204D1099D49004B5B00E00023311F6B
:108A50000024095F0E9D1202491BCC1709196140C1
:108A60005943059D6D18B11E0024095F05958A1AAA
:108A7000D51752196A405343049C069AE41804948B
:108A80009FE79C4692E7331F1A78B31E1B78802A13
:108A900002DD802149008A1A802B02DD80214900F5
:108AA000CB1AD3180693294B06981B681A1C7332ED
:108AB00011787E330132FEF74FFD254B041C1B68F5
:108AC0000022B05E1425595F5A6A40231B1B009395
:108AD0000023FEF718FD2318049C05985C430494BA
:108AE0000025745F5843A501291CF7F7C3FD291C15
:108AF00005900498F7F7BEFD011C0598FFF704FEEA
:108B000014497080CA7880B212907F208243042377
:108B10004B701343802252421343069DCB701220A8
:108B2000B02310AA1097119513940B71FEF7C0FB98
:108B3000013F0E3E24E715B0F0BDC046C003002043
:108B4000C8030020BE990000C69900007C090020DF
:108B500078090020EF0100204C4BF0B51B6885B070
:108B60005A681D6A013A120202920E241A686B1E9C
:108B70005C43013A0419019012020020039204346C
:108B80000090002D68D0424F3B681A1C493216787D
:108B9000012E17D10022A15E1A1C4A32128891427E
:108BA0000EDD4C3362881B789A4209D93949267206
:108BB000B5230E2000220B71FEF77AFB009601E030
:108BC000002323723E68331C4D331B78012B40D1A8
:108BD0000023E25E331C50331B889A4239DD231F89
:108BE00000201A5EFF2A0ADDA31E00215B5EFF2B18
:108BF00005DD0298824202DC03998B4229DA264B7A
:108C000005211A6804236156E356D06BCB1A1B0268
:108C100043430621072020566156926B411A0902F0
:108C200051431B1409140A208B4201DB584301E015
:108C30004843191CF7F71EFD4E363378984208DD7D
:108C40000123144923720E20B62300220B71FEF774
:108C50002FFB013D0E3C94E70099002913D00B4BEC
:108C60000E221B6801981B6A5A438218013B0AD3E3
:108C7000111C0A390020095E002902DD911E012025
:108C800008700E3AF2E705B0F0BDC046C003002000
:108C900078090020CB040020C8030020F0B51E4B4B
:108CA00085B01B6803911B6ADBB2013BDBB2FF2B73
:108CB00030D0039CD900611804254E5F0E249D001E
:108CC000002E1FD05C4304190427E65F5519002EBF
:108CD00014D02688019535B2AC4600254F5F654615
:108CE000ED1B6F10BE19019F3E8064880225495F0D
:108CF00026B2711A49100C197C80D6E70C882C809A
:108D0000498805E05C430419218855192980618848
:108D10006980CAE705B0F0BDC0030020F8B5124C69
:108D2000051C20680A222830002100F095FD0F4B19
:108D300020681B681A6AD2B2013AD2B20023FF2A15
:108D40000DD00E215143862769188B80BF008118F2
:108D5000CE1933718826B60089198B71ECE7226829
:108D600013645364F8BDC046C8030020C00300204C
:108D7000704700000F4AC378126810B551685CB2A2
:108D800001398C4201DA0133C370837859B200296A
:108D900001DD013B83704378126859B2013A914278
:108DA00001DA0133437003785AB2002A01DD013B36
:108DB000037010BDC0030020F0B5BA4D8BB007930F
:108DC0002B6805920C1C5A68B749049018684A70C1
:108DD0009A68059E8A70012301320870CB70B21820
:108DE000082306200B71FEF763FA2B68DB6ADBB2FF
:108DF000013BDBB2FF2B09D0049F1A01BA187F2177
:108E000091721173FF21D1725173F1E7A74B0022C8
:108E10001B68119D1A600922AA56119D0823EB5662
:108E20009A4256DB119E0B217156119F0A23FB5665
:108E300099424CDB9B4B501C1E68B768F66A78431E
:108E4000059F013040183D182B78B34204DD3E2BBE
:108E50003BD800232B7038E0002B36D0109D40000B
:108E6000405B924D013B2D682E6801362E60049EBA
:108E7000DDB22B01F318061C4E431F68BE191E609D
:108E8000061C56435F68BE195E601E8986191E81E6
:108E90000C269E57B14200DA19730D269E57B14237
:108EA00000DD59730A269E57B24200DA9A720B26E9
:108EB0009E57B24200DDDA72AD0065190026AB5F45
:108EC000834202DA2880EA70A9700139ADE7013ADD
:108ED000A3E70026049F0696724E069C3368DB6A61
:108EE0009C4200DBE8E008203B5E002B00D1E3E081
:108EF000381C0A300B24FFF73DFF3C5701940A232E
:108F0000FB56019D9D4200DAC6E00D257D57039575
:108F10000C23FB56039E9E4200DABAE0614B039C91
:108F20001E68019BB06801334343059D01331B1943
:108F3000ED182A7800900295002A02D03F2A00D02E
:108F4000A4E0109D5B005C5B002C00D19EE0002340
:108F500009930523013B002B26D0554A0125D21841
:108F60006D425557534A0121D21849425156019832
:108F7000009A411801314A430598039994464218D2
:108F80005219624451780029E4D0F26A9142E1DC3E
:108F9000002209A8855C002D01D18154DAE78D42B9
:108FA000FBD00132D2B2F4E709AA9A5CDDB2002A02
:108FB00004D00133042BF7D11D1C01E0002D65D036
:108FC000291C201CF7F756FBF16A029E0131491952
:108FD0003170039E002246430096019E464302964E
:108FE0006B1E9C4609AB9B5C049E013B1B01F31866
:108FF000624513DA1E68241AB446009E0132B44456
:1090000066461E605E68B446029EB44466465E6074
:109010001E89B446844466461E81E1E7039A1868B7
:10902000624382181A60019A5E686243B2185A60FD
:109030001A89A4181C811B4B1B681B6B994225DDE8
:109040000023634522DA01331A1CAA42F9DA09A87F
:10905000C11801390978105C01390138C9B2C0B2B0
:109060000124814208D2079E890071188440201C87
:109070000C682043086007E0079E800030188C4091
:10908000211C0468214301600132DEE7039D013D9C
:109090003DE7019C013C31E7069E103701360696FC
:1090A0001AE7C046C0030020C4040020C803002003
:1090B000BE990000C699000000253368DC6AA5420D
:1090C00005DA049F2C013C192789002F15D1154A78
:1090D00015491268186815645A68059C4A709A68A0
:1090E00001238A7001320870CB70A2182D2306204C
:1090F0000B71FEF7DDF80BB0F0BD21683FB208023E
:10910000391CF7F7B7FA62682060391C1002F7F7CC
:10911000B1FA6060201C0A300135FFF72BFEEDB27A
:10912000CBE7C046C8030020C4040020F0B5544A71
:10913000544B12681B6811791A2251438BB059188D
:1091400003AD1831041C281C00F044FB4E4B0021D9
:109150001B6800915A681F68013A1202013F019290
:109160003F02494E009933681A6A914200DB84E05D
:109170000421625E002A7BDD414A12681279012ACD
:1091800076D00022A05EFF2817DC0533DB7F6A461D
:1091900029780D32002B01D007AB01E06B4612336A
:1091A000FEF7DAF90021635E00B2013BFF3B584352
:1091B00080110130FF3020801FE0019A101AFF2833
:1091C0001BDC0533DB7F6A4629780D32002B02D089
:1091D0006B46213301E06B461733FEF7BDF90021E2
:1091E000625E019900B28A1A013AFF3A5043019B2C
:1091F0008011013BFF3B1B1A23800222A05EFF2847
:1092000018DC33686A460533DB7F29780D32002B82
:1092100002D06B46173300E007ABFEF79DF9022141
:10922000635E00B2013BFF3B584380110130FF30C9
:1092300060801DE0381AFF281ADC33686A4605335F
:10924000DB7F29780D32002B02D06B46123301E010
:109250006B462133FEF780F90221625E00B2BA1A32
:10926000013AFF3A50437B1EFF3B80111B1A63807B
:10927000009A0E340132009273E70BB0F0BDC04685
:10928000C80300207C090020C0030020F8B5124E5E
:10929000041C33680D1C0633DF7FFEF769F80F4BA3
:1092A0001B68D4331B781840336878405A1DD27F2E
:1092B000002A07D02288298821802A80002809D006
:1092C0001B6802E0002805D05B682288013B1B0276
:1092D0009B1A2380F8BDC046C00300207001002007
:1092E000F0B5038887B005AD00902B8043886946B0
:1092F0001631281C0B80FFF7C9FF2D4B1A68531D30
:10930000DB7F81CA2B4A002B03D0411E0902013F9B
:1093100002E0013F3902471E12683F029368D66897
:10932000254A02971468226801920022A85E019AD9
:10933000C0185B00C9185043F7F79CF980B2288029
:109340006D46163503900021685E029A67688019A1
:10935000760091197843F7F78DF9164986B20968B6
:109360002E80231C0979663367341A782378022902
:1093700001D101231A1C039C05A920B2904206DDED
:10938000019CA41AA04203DB01980138821A0A80CA
:1093900036B29E4204DDFA1A964202DB7A1ED31AD6
:1093A0002B800B88009C23802B88638007B0F0BD46
:1093B000C0030020C80300207C090020034B822248
:1093C0001B6892009B1858687047C046C80300206D
:1093D00038B5041C081C002A07D0D1185843624332
:1093E0004D1010184019F7F745F938BD10B5F7F7CB
:1093F0006BFA064B01781C68054B1B68586BF7F736
:10940000EBF8C6239B00E05010BDC046C803002007
:1094100078090020014B18607047C0468009002081
:10942000F0B58BB0041C101C11AA12781F1C9446B6
:1094300010AB12AA1B7812785D4D059304922B682D
:109440002A680E1C0421515E06229A5E6346009330
:10945000059BFEF758F8391C8002F7F70BF92F68C7
:1094600005903A787300002A00D191E0514A1168C2
:10947000B02252008A5C022A00D189E07A78F11C7D
:10948000002A19D14A00A218111C083909889C46E3
:109490001180911F0888911E08806189584261805F
:1094A000218909902180B11C49006518083961188B
:1094B00007950891331C37E0B01C00224000628001
:1094C0002280049D22522018428049005842321CBA
:1094D00064186E00049058E003217956951E03919C
:1094E000911F0888298806954018099D03994843CB
:1094F0005119614408390D8811886918049D694320
:10950000151F4118022038562D8868430818059900
:109510008011484300141080721E934207D1089DA9
:1095200007982A880280069A013BD5D23DE0012B9C
:10953000F9D1E2886280F6E703203856A11F400087
:109540008446A01E05880988081CA94200D2281C50
:1095500080B261464143049D8C466119C91808399F
:109560000D882088291C854200D2011C251F02205D
:1095700038562D8889B271436843614409180598AB
:109580008911414309142180023C013AD4D20CE0F4
:10959000E4180022964208D05100611A4B88059DBC
:1095A00001326B431B14CB80F4E70BB0F0BDC04617
:1095B0008009002070010020014B18687047C046E8
:1095C000880900209120C00070470000024B1868F5
:1095D0008C239B00C018704788090020F42358434F
:1095E000A8239B00C018024B1B6818187047C04680
:1095F000880900206A23FF335843014BC018704785
:1096000098B4000000487047D3B8000010B5FBF7CD
:10961000AFFC0F4B41791B685960427902329A6066
:1096200082791A604A43DA604179042299610479A7
:10963000002C00D002225A614A43DA6102681A62A1
:1096400001795A1DD17702790633DA7710BDC04609
:10965000C003002010B51248124C2060FBF782FCBA
:109660002068B030F7F71EF920680130FF30FDF7B1
:109670008BFF20681130FF30FEF73AFC20688B2307
:109680009B00C018FDF7A0FBFFF7C0FF064C201C95
:10969000FBF780FC054BE018FDF78EFF10BDC046C0
:1096A00010B000008809002098B400006B0400008E
:1096B00010B5FBF75DFC114B81791B68596082790D
:1096C00002329A6042791A604A430D49DA600A1CF4
:1096D0003C32807912780C1C98610421002A00D059
:1096E000022159614143D961211C3D310978196238
:1096F000591D0633CA77DA7710BDC046C003002073
:1097000010B0000008B5FFF7D3FF0248FBF742FC9A
:1097100008BDC0466AB7000038B5124BF4241B6878
:109720001B785C43A8239B00E4180F4B1B681C1993
:10973000251C0E4BE835201C1C60FBF71FFC281C69
:10974000FFF768FE201C7030F7F7B8F8201C78305F
:10975000FDF726FF201C8830FEF7D6FB281CFDF7FE
:1097600039FB38BDCC030020880900208409002083
:10977000014B1B6818707047CC030020014B1B681D
:1097800018787047CC03002000487047A4B300004D
:1097900000487047B0B20000F8B50D1C041C081C4E
:1097A000111C161CF6F766FF311C071C281CF6F767
:1097B000B7FF002D05DB002908DB2760201C616056
:1097C000F8BD0029F9DD013F8919F6E70137891B4A
:1097D000F3E7C046F0B50F2A35D9031C0B439C07AD
:1097E00035D1161C103E36093501451910350C1CB3
:1097F000031C27681F6067685F60A7689F60E76851
:109800001034DF601033AB42F3D1731C1B01C51859
:10981000C9180F231340032B1BD91C1FA4080134A4
:10982000A4000023CE58EE500433A342FAD1ED1821
:10983000C91803231A4005D00023CC5CEC54013333
:109840009342FAD1F0BD051C002AF5D1FAE7051CB8
:10985000F2E71A1CF8E7C046F0B5830746D0541E5D
:10986000002A42D0CEB2031C032503E0621E002C66
:109870003BD0141C01335A1E16702B42F6D1032C18
:109880002BD9FF250D402A0215432A0415430F2C1E
:1098900015D9271C103F3F091E1C3A011036B61877
:1098A0001A1C156055609560D5601032B242F8D12F
:1098B00001373F010F22DB191440032C0DD9271F5C
:1098C000BF08BA001E1DB6181A1C20C2B242FCD135
:1098D0000137BF000322DB191440002C05D01C19EE
:1098E000C9B219700133A342FBD1F0BD141C031C93
:1098F000C5E7C046AAAAAAAA5555555500000000BA
:10990000FFFFFFFF0201000200010001020010271B
:109910005E0E4905F101B700430018000100000088
:1099200050CCCC504199994150CCCC94429999500B
:1099300050CCCC15409999544099999502333354A1
:109940000600000008000000000000000B000000FE
:1099500002000000070000000900000000000000F5
:109960000C0000000300000000007804EF08660D02
:10997000DB115016C21A331FA1230C28742CD930C6
:1099800039359639EE3D42429046D94A1B4F5853DD
:109990008E57BE5BE65F07641F68306C39703874A1
:1099A0002F781C7CFF7FD983A8876D8B278FD5925A
:1099B0007996109A9B9D1BA18DA4F3A74BAB97AEF4
:1099C000D4B104B526B839BB3EBE34C11BC4F2C6FF
:1099D000BAC973CC1BCFB3D13BD4B2D619D96EDB85
:1099E000B3DDE6DF08E218E416E603E8DDE9A5EBFF
:1099F0005BEDFEEE8FF00DF277F3CFF414F646F741
:109A000064F86FF967FA4BFB1BFCD8FC81FD17FE6D
:109A100098FE06FF5FFFA5FFD7FFF5FFFFFF00FFE2
:109A20000100FFFF0101FF000001FF01FF01000134
:109A30000203040405060708090A0B0B0C0D0E0FA0
:109A4000101111121314151516171818191A1B1BBB
:109A50001C1D1D1E1F1F20212122232324242525F8
:109A6000262727282829292A2A2B2B2C2C2D2DFF85
:109A700000000000000000000000000000000000E6
:109A800000000000000000000000000000000000D6
:109A900000000000000000000000000000000000C6
:109AA00000000000000000000000000000000000B6
:109AB00000000000000000000000000000000000A6
:109AC0000000000000000000000000000000000096
:109AD0000000000000000000000000000000000086
:109AE0000000000000000000000000000000000076
:109AF0000000000000000000000000000000000066
:109B00000000000000000000000000000000000055
:109B10000000000000000000000000000000000045
:109B20000000000000000000000000000000000035
:109B30000000000000000000000000000000000025
:109B40000000000000000000000000000000000015
:109B50000000000000000000000000000000000005
:109B600000000000000000000000000000000000F5
:109B700000000000000000000000000000000000E5
:109B800000000000000000000000000000000000D5
:109B900000000000000000000000000000000000C5
:109BA00000000000000000000000000000000000B5
:109BB00000000000000000000000000000000000A5
:109BC0000000000000000000000000000000000095
:109BD0000100000000000000000000000000000084
:109BE000000000200400000031190000951A000058
:109BF000B51A0000C51B0000FD1B0000131C00006F
:109C0000291C0000811C0000D91C0000031D00005D
:109C1000391D00008D200000DD1E0000DD1E00004B
:109C20000000000000000000112B0000ED2F0000DC
:109C300000000000A5200000A920000099210000DC
:109C4000B9210000F1210000612400003D2900003D
:109C500019340000EC03002001030084000000011F
:109C60000000000000004D49500000000000040505
:109C7000004D3448304D4500000005000001000152
:109C800000000000000000000000000000000000D4
:109C9000000000000000000000000000D3040020CD
:109CA00007000000980500209002002070050020A9
:109CB00002000000002010026A08060000201002C6
:109CC0001E00010000200102010000000000010050
:109CD000203040507000102004050700F4020020DE
:109CE0006502002068020020030000000700000059
:109CF0002C020020DE0400207C0200200100000075
:109D000000200060FF000001001011001020303121
:109D100008012001040000000000000048030020AA
:109D200058030020000000000000000000000000B8
:109D30006C03002000000000000000000000000094
:109D40008403002000000000300300200000000019
:109D500000000000000000006C0200200000000075
:109D60008002002054020020580200200000000061
:109D70005D020020DA04002000000000EB04002057
:109D8000F2040020F3040020780500200000000009
:109D900000000000DF040020F60100200002002087
:109DA000A00300209B020020A0020020050000006C
:109DB0001D08080C0A0A0000180300205F0200209A
:109DC00040030020060000000C0300209802002041
:109DD000300200200300000000100220B403002025
:109DE000680300206A030020020000000010200821
:109DF00002200000940300207C0300207F03002049
:109E00000300000044020020940200200000000033
:109E10004C020020D20400200000000000000000DE
:109E2000000000000A0200200C0200200D141B009C
:109E3000AC050020E0050020FC05002018090020EA
:109E4000FFFFFFFFFFFFFFFFFFFFFFFFFFFFFFFF22
:109E5000FFFFFFFFFFFFFFFFFFFFFFFFFFFFFFFF12
:109E6000FFFFFFFFFFFFFFFFFFFFFFFFFFFFFFFF02
:109E7000FFFFFFFFFFFFFFFFFFFFFFFFFFFFFFFFF2
:10B05000FFFFFFFFFFFFFFFFFFFFFFFFFFFF0400FA
:10B060004D34483050415241303030303030303043
:10B070000A00000001180E00010000000102030494
:10B0800005060708090A0B1A1B1C1D1E1F2021227A
:10B09000232425191817161514131211100F0E0D4D
:10B0A0000C00000000000000000000000001000093
:10B0B000BF00F000000000000000000000000000E1
:10B0C00000000000000000000000000F0000000071
:10B0D00000000000BF00F0000000000000000000C1
:10B0E0000000000000000000000000000000000F51
:10B0F00000000000000000008300000040033F2229
:10B100008000000000033F28230303080000170A03
:10B110000400020101002C012C012C012C01000073
:10B120004A375F44554F0000000000000000000057
:10B13000323205040600FFFFFFFFFFFFFFFFFFFFA6
:10B140000A05BC02B6032C012C015000FFFFFFFFD3
:10B150001E1E14000300F401F6FFFFFF0A000000AA
:10B1600010283C00FFFFC800B80B1E0001000000C3
:10B17000140005004000030C280000800100760246
:10B18000D0020000000500000100000001000000E6
:10B19000010000000100000005004080C4FF62566D
:10B1A0004E464062564E464060544E4640645A50A9
:10B1B0004B41000000000000000000000000000003
:10B1C000000000000000000000000000020040003D
:10B1D000000080800000008080000000808000006F
:10B1E0000080800000000A0AAB02BE043C004B0055
:10B1F0009001010600417E99D6F30000000031293C
:10B2000026231F1E000000000102CA031E005A0070
:10B210005A000A008E035A005A000A001E00160344
:10B220005A000A001E005A0016034006FA004006A3
:10B23000FA004006FA004006FA000001020101008F
:10B2400000010100000190010001409C00019001FB
:10B2500000000000C8004B063000B0043200F401CA
:10B260000100321EE6003704E001EB049D008D0072
:10B270005B003A00300000000100000005000A00F9
:10B280000F0014001E002800000000002800280005
:10B29000280028002800280000000000010000000D
:10B2A000B200F000000000000000000000000000FC
:10B2B00000000000000000000000000F000000007F
:10B2C000000000008000000040033B18D100007126
:10B2D0000A48F61C002D0F052D0F052D0F05000047
:10B2E000000000000000000000000000000000005E
:10B2F000000000000000000000000000000000004E
:10B30000000000000000000000000000000000003D
:10B31000B200F0000000000000000000000000008B
:10B3200000000000000000000000000F000000000E
:10B33000000000008000000040033B18D1000071B5
:10B340000A48F61C002D03032D03032D0303000000
:10B3500000000000000000000000000000000000ED
:10B3600000000000000000000000000000000000DD
:10B3700000000000000000000000000000000000CD
:10B38000785AF0001E03D8FF010000005A030A009B
:10B3900000800A0A0A0CF9000500000000000E00F7
:10B3A000140019001A0000000000000038003800E6
:10B3B000500078007800000000000000C00100008C
:10B3C00050A0B003520326025E0130001027000097
:10B3D00002010100000000000F0000000F01011435
:10B3E0000000080769001900FA000613133D8002E7
:10B3F000000120005A00000001000A0D1C003C0062
:10B4000008100810B200F00000000000000000006A
:10B410000000000000000000000000000000000F1D
:10B42000000000000000000080000000400303183E
:10B43000D10000710A48F61C00371B05371B053781
:10B440001B050000000000000000000000000000DC
:10B4500000000000000000000000000000000000EC
:10B4600000000000000000000000000000000000DC
:10B4700000000000785A90000A03D8FF0100000085
:10B480005A030B0000800B0F0A0CF90005000000A6
:10B4900000000E00140019001A0000000000000057
:10B4A00038003800500078007800000000000000EC
:10B4B000C001000050A04C03EE02C201FA003000AF
:10B4C0001027000002010100000000000F00000032
:10B4D0000F0101140000080769001900FA000613A3
:10B4E000133DE402000124005E0000000100060D8F
:10B4F00028005000172B172B080809090A0A0A0A06
:10B500000B0B0C0C0D0C0D0D0D0D0D0D0D0D0D0D72
:10B51000080809090A0A0A0A0B0B0C0B0D0D0D0D80
:10B520000D0D0D0D0D0D0D0D080809090A0A0A0A69
:10B530000B0B0C0B0D0D0D0D0D0C0D0D0D0D0C0D44
:10B5400008080809090A0A0A0A0B0B0C0C0D0C0D55
:10B550000D0C0D0D0C0D0D0C0708080909090A0A40
:10B560000B0B0B0B0C0D0D0C0D0D0C0D0D0C0D0D17
:10B57000070708080909090A0A0A0B0B0C0C0C0C2E
:10B580000C0C0C0C0C0C0C0D070708080909090918
:10B590000A0A0B0B0C0C0B0C0C0B0C0C0C0C0B0DF3
:10B5A0000607070808090909090A0A0B0B0B0B0B08
:10B5B0000C0B0B0C0B0B0C0B0607070808080809F3
:10B5C000090A0A0A0B0B0B0B0B0B0B0C0B0B0B0BCF
:10B5D0000606070708080808090909090A0A0A0BE4
:10B5E0000B0B0B0B0B0B0A0B0606060707080808CC
:10B5F000080909090A0A0A0B0B0A0B0B0B0B0B0BA8
:10B600000506060707070708080909090A09090ABC
:10B610000B0B0A0B0B0A0B0B0505060607070707A2
:10B62000080808090909090A0A0A0A0A0A0A0A0B83
:10B630000505050606070707070808090909090A95
:10B640000A090A0A090A0A0A0000000000000000AC
:10B6500000000000000000000000000000000000EA
:10B6600000080809090A0A0A0A0B0B0C0C0D0C0D3C
:10B670000D0D0D0D0D0D0D0D0D080809090A0A0A15
:10B680000A0B0B0C0B0D0D0D0D0D0D0D0D0D0D0DF4
:10B690000D080809090A0A0A0A0B0B0C0B0D0D0DFF
:10B6A0000D0D0C0D0D0D0D0C0D08080809090A0AE9
:10B6B0000A0A0B0B0C0C0D0C0D0D0C0D0D0C0D0DC9
:10B6C0000C0708080909090A0A0B0B0B0B0C0D0DD6
:10B6D0000C0D0D0C0D0D0C0D0D07070808090909BF
:10B6E0000A0A0A0B0B0C0C0C0C0C0C0C0C0C0C0CA2
:10B6F0000D07070808090909090A0A0B0B0C0C0BAE
:10B700000C0C0B0C0C0C0C0B0D0607070808090998
:10B7100009090A0A0B0B0B0B0B0C0B0B0C0B0B0C7C
:10B720000B0607070808080809090A0A0A0B0B0B89
:10B730000B0B0B0B0C0B0B0B0B0606070708080873
:10B7400008090909090A0A0A0B0B0B0B0B0B0B0A58
:10B750000B0606060707080808080909090A0A0A65
:10B760000B0B0A0B0B0B0B0B0B050606070707074A
:10B7700008080909090A09090A0B0B0A0B0B0A0B2D
:10B780000B05050606070707070808080909090940
:10B790000A0A0A0A0A0A0A0A0B0505050606070725
:10B7A00007070808090909090A0A090A0A090A0A09
:10B7B0000A0000000000000000000000000000007F
:10B7C0000000000000000000000005060606070754
:10B7D00007080909090909090606060707080809EB
:10B7E000090A0A0A0A0A06060707080809090A0ACE
:10B7F0000A0A0A0B0707070808090A0A0A0B0B0BB3
:10B800000C0C07070808090A0A0B0B0B0C0C0D0D92
:10B81000070809090A0A0B0B0C0C0D0D0D0D080980
:10B82000090A0A0B0D0D0D0D0E0E0E0E09090A0A5E
:10B830000C0C0C0D0D0D0F0E0E0E090A0A0B0D0D42
:10B840000D0E0E0F0F0F0F0E090A0C0B0D0E0E0E24
:10B850000F0E100F10100B0C0C0D0E0E0D100F1103
:10B860000F110F100B0C0C0C0D0E0F0F0F0F1010F3
:10B8700011100C0C0D0E0E0F1011111110111212CF
:10B880000C0C0C0D0F0F0F111010111111110C0DCC
:10B890000D0E0F100F101111111111120B0C0C0DB8
:10B8A0000E0F0F111011101112110C0D0E0E0F10A2
:10B8B00010101112111212120D0D0C0E0F0F10118B
:10B8C0001011111211120D0D0E0F0F0F1011111278
:10B8D000121112110D0C0F0F0F1011111011121265
:10B8E00012120C0D0D0F0F0F10111111111111115A
:10B8F0000C0D0E0F0F0F10111111111212120D0D50
:10B900000E0E0E0F0F0F1011111211120E0E0F0F3F
:10B910000F0F11111111111313130000000000007B
:10B920000000000000000000000000000000000017
:10B9300000000005050506060707070708080909AE
:10B9400009090A0A090A0A090A0A0A0E0E0F0F0F44
:10B950000F1111111111131313000000000000004A
:10B960000000001F23232527282A2B2D2E2E2F31C0
:10B970002F3333333533333535363C1C1E1F2123EB
:10B98000242626272828292B2B2B2D2D2D2E2D2E16
:10B990002F2E331D1F202323242527282929292A38
:10B9A0002C2C2D2F2E2D2F2E2E2F341D1E212123FA
:10B9B000232626262A2A2B2B2C2D2C2C2F2E2F31DA
:10B9C000302F341E1E21222325262828282B292902
:10B9D0002C2C2D2E2E2E2E2E302F351E1E212222C7
:10B9E0002525252829292A2A2D2D2D2F2F2D2F30A9
:10B9F0002E30341D1F20222424262627292A2B2BD3
:10BA00002D2D2C2F2F2D2F302F2E331D1E21222494
:10BA100023262626282A292A2D2D2D2D2F2E2E2E7F
:10BA2000302F331E1D2020222425262827292A2BAB
:10BA30002C2D2D2F2F2E2E303030341E1E1F212363
:10BA400024262628292B2B2B2D2E2E2E302E2E2E43
:10BA5000302F331E1E2122242525262728292C2974
:10BA60002D2E2B2F2F2D2F2F2F31311D1E2020213A
:10BA70002424262728282B2A292C2D2C2E2E2D2E27
:10BA80003030341D1D202122232425262728282A52
:10BA90002B2A2C2C2C2D2E2D302F2F222124252704
:10BAA00028292A2B2C2D2D2F3031333331333332AB
:10BAB00034363500000000000000000000000000E7
:10BAC0000000000000000000000000001E212326EE
:10BAD00029282B2F2E2F2F2F2F3131323434363768
:10BAE0003837383B1C1E2022242626282A2C2C2DB1
:10BAF0002B2D2E2E3030302F313334351D1E212288
:10BB00002527282B2A2A2C2D2D2C2D2F3130313171
:10BB1000333433351D1E21222726292B2B2B2D2D87
:10BB20002D2C2F2F31303132313534351E1E21234B
:10BB30002628292B2B2D2D2F2D2E2E2F2F33323132
:10BB4000333333371E1F2223232828292B2C2F2F52
:10BB50002F2E2F2F30313331323333371E1F222215
:10BB60002326282A2A2C2C2E2E2F2E31322F313309
:10BB7000333633371E1E21222426282A2A2A2E2D28
:10BB80002F2E2E312F2F3433313435351E1E2123E5
:10BB900024252828292A2C2D2E2F2F312E313235DD
:10BBA000353334361E1F21232525292B292C2D2EF4
:10BBB0002D2E2F3031333133333433381E1E2022B3
:10BBC00024252629292A2C2D2C2F2E2F2F333333B1
:10BBD000333534381E1E202224252726292B2C2CD1
:10BBE0002A2C2F3131313334323333351C1D1F2190
:10BBF00023232527282C2C2B2B2C2D2C3030313295
:10BC0000313332351F1F24242627282D2E2F303183
:10BC10002E323135353335373535353800000000B3
:10BC20000000000000000000000000000000000014
:10BC300000000000001F20242628282A2D2C2E2F4B
:10BC40002F2D2F3230333333353335353A1E1E2105
:10BC5000232526262729292A2A2B2C2C2D2D2E2E4A
:10BC60002F312E31361E1E212226262728282A2A49
:10BC70002A2C2B2B2E2D2C2F2F303131331E1E2111
:10BC800023242729282A292B2C2D2C2D2C2F2F2F0C
:10BC900030303433351D1F202425262928292B2B0D
:10BCA0002B2D2D2D2D2E2E2F312F3131341E1E21D7
:10BCB00023252626282A2A2B2C2D2D2B2F2E2D2FDF
:10BCC0002E303233371F1E222325262728282A2CE0
:10BCD0002D2E2E2C2E302F3130313331381E1F2196
:10BCE00024232728282B2A2B2D2D2C2F2F2E312FA4
:10BCF00031333331381E1E2123242426282B292BAF
:10BD00002F2D2D2F2C30313131323231381E1E2162
:10BD100024242627282B2A2B2B2C2D2F2E2F2F3275
:10BD200031323331361E1E2124252727282B2B2A7A
:10BD30002C2C2D2E302F2F3232313230381E1E2037
:10BD40002225252729292B2C2C2B2C2E2E31313046
:10BD500033313132371D1D2122242624262A282A58
:10BD60002B292B2B2C2D312F3130313138201E2116
:10BD700024252828292B2D2E2E2C2D303031313101
:10BD800034343233350000000000000000000000B1
:10BD90000000000000000000000000000000FFFFA5
:10BDA000FFFFFFFFFFFFFFFFFFFFFFFFFFFFFFFFA3
:10BDB000FFFFFFFFFFFFFFFFFFFFFFFFFFFFFFFF93
:10BDC000FFFFFFFFFFFFFFFFFFFFFFFFFFFFFFFF83
:10BDD000FFFFFFFFFFFFFFFFFFFFFFFFFFFFFFFF73
:10C01000FFFFFFFFFFFFFFFFFFFFFFFFFFFF04002A
:10C020004D4254014D3448300000000000C0000073
:10C03000EEEE090604000400EEEEEEEE002C2C30CD
:10C04000002201010010000008031820300718002A
:10C0500000000000000000000000400028B50000C3
:00000001FF
